:020000040800F2
:2000000000500020197F0008617F0008617F0008617F0008617F0008617F00080000000048
:20002000000000000000000000000000617F0008617F000800000000617F0008B7660008E3
:20004000617F0008617F0008617F0008617F0008617F0008617F0008A9680008AF680008F8
:20006000B5680008BB680008C1680008617F0008617F0008617F0008617F0008617F000877
:20008000617F0008617F0008617F0008617F0008617F0008617F0008617F0008C7680008D1
:2000A000617F000809640008617F00081D640008216400083564000849640008B1310008A5
:2000C000BD310008C9310008D5310008617F0008617F0008757500088D750008A975000828
:2000E000EF680008617F0008617F00080000000000000000000000000000000000000000D1
:2001000000000000000000005FF808F1034613F8012B002AFBD1181A0138704710B5054CE1
:20012000237833B9044B13B10448AFF300800123237010BD0801002000000000348D000841
:2001400008B5034B1BB103490348AFF3008008BD000000000C010020348D0008704790F914
:200160002C30002BBABF90F82900C00900207047024690F82C3013F040001CBF92F8290031
:20018000C0F380107047024690F82C3013F020001CBF92F82900C0F340107047024690F8FE
:2001A0002C3013F010001CBF92F82900C0F300107047024690F82C3013F008001CBF92F82C
:2001C0002900C0F3C0007047024690F82C3013F004001CBF92F82900C0F3800070470246D9
:2001E00090F82D3013F010001CBF92F82A00C0F300107047024690F82D3013F008001CBFEB
:2002000092F82A00C0F3C000704700000122014B1A707047C303002010B50446034B0449C0
:200220000360044807F01FFD204610BDC89500084C8D0008F406002010B50446FFF7ECFF79
:200240002046302106F061F9204610BD012A02D1016000207047022A05D0032AF9D0002A0D
:20026000F7D10260F5E70B680360F2E703681847012A02D1016000207047022A05D0032A9B
:20028000F9D0002AF7D10260F5E70B680360F2E7036808681847836810B5044613B1032299
:2002A00001469847204610BDCBB2322B08D80E4A01F4E06152F823301943C0F8881070479D
:2002C00001F0C002C02A0CD1CF2B0AD8074B01F03F0253F82220044B01F4E06153F8223095
:2002E000EAE74FF0FF31E8E7289C0008E89B0008CBB2322B08D80E4A01F4E06152F82330B3
:200300001943C0F88410704701F0C002C02A0CD1CF2B0AD8074B01F03F0253F82220044BC8
:2003200001F4E06153F82230EAE74FF0FF31E8E7289C0008E89B0008036810B51B6B044684
:2003400098474A2808D10423237123682046D3F8E0309847012010BD0020FCE770B5067B76
:20036000044616B1FFF7E8FF70BD012303730369ABB1D0E905230B490B4807F074FC206988
:2003800002F012FAD4E904512846FFF7B1FF2846A169FFF789FF3146284602F091FC204679
:2003A000E0E700BF5C8D0008F406002038B52C2007F0F6FE01280446084D0CD12B78012B14
:2003C00003D00749074807F03BFC00210E2007F0ADFE2C7038BD0121F8E700BFC003002058
:2003E0006A8D00087402002010B5064B42F210705C7907F0C9FD2146BDE81040082007F091
:20040000C9BD00BF2401002038B5074D6C79044484F3080442F2107007F0B6FD2146082074
:2004200007F0B8FD6C7138BD2401002070B50A4EB47A0444A4F11403EB2B254684BF002571
:200440002C4642F2107007F09FFD2946282007F0A1FDB47270BD00BF2401002070B50E4AC3
:200460000E4913780E4E013303F00303CC5C1370B27A42F210701444A4F11403EB2B254601
:2004800084BF00252C4607F07FFD2946282007F081FDB47270BD00BF5C0200200000002033
:2004A0002401002000212D2007F040BE01212D2007F03CBE70B505460C460026AE4205DB7C
:2004C0002146BDE870402D2007F030BEFFF7EAFF4FF4C87007F0A4FEFFF7E8FFC82007F07F
:2004E0009FFE0136EAE700000022044B83F8402083F83F2083F83E20704700BF14020020AC
:200500000F4982B0ADF8040091F83E001E2815D891F84030BDF80420013021F813201F221E
:200520000133DBB2B3FBF2F281F83E000120C2EB42129B1A81F8403002B070470020FBE786
:200540001402002007B5ADF804000198FFF7D8FFD8B90F49BDF8042091F8403021F8132093
:200560001F220133DBB2B3FBF2F0C0EB40101B1A81F8403091F83F300133DBB2B3FBF2F285
:20058000C2EB42129B1A81F83F3003B05DF804FB1402002037B5144B1B7823B903B0BDE86E
:2005A0003040FFF7A1BF114C8DF80400A5788DF80510EB0642BFE37843F00803E370019861
:2005C000FFF79EFF68B9AA0742BFE37843F00103E370EB0705D5019803B0BDE83040FFF7AD
:2005E000B1BF03B030BD00BFC10300202401002037B5104A92F83E30D3B192F83F40013BFC
:20060000611CC9B282F83F1012F8140002EB440465781F24B1FBF4F482F83E302B46C4EB0A
:200620004414091B82F83F1040EA032003B030BD1846F9E71402002038B50024114B124D48
:20064000C3F8D440A3F8D840022115F8010B013407F00EFD072CF7D100240C4D002115F8FF
:20066000010B013407F004FD082CF7D10024084D022115F8010B013407F0FAFC0C2CF7D16E
:2006800038BD00BF34010020A0970008989700088C97000808B507F083FD003818BF01204C
:2006A00008BD0000D222064B9A700A229A710522DA71FF225A7100229A72DA72704700BFA1
:2006C000240100202DE9F041D0F814E004460F4616461D46BEF1000F04D0F446BDE8F041D2
:2006E000007C6047406818B94FF0FF30BDE8F081217C02F09BF86068394603681B689847A4
:20070000606802F018FA0028EED12A46217C606802F00EFA60682A4603683146DB6998471A
:20072000281A18BF4FF0FF30E0E7002307B58DF807300DF107020123FFF7C4FF431C18BFB6
:200740009DF8070003B05DF804FB10B51446FFF7ECFF431C0ED0C117C4F12002A4F1200352
:20076000E04001FA02F2104321FA03F3184300F0010010BD0020FCE708B5032200210C30AB
:20078000FFF7E3FF08BD10B500F10C04012103222046FFF7DAFF014620B905222046FFF7D7
:2007A000D4FF10BD0020FCE708B5142931D8DFE801F00B11131517303030303030191C1E0D
:2007C00020222426282B2E00002280210C30FFF7BCFF08BD0122F8E70222F6E70322F4E794
:2007E0000422F2E700229021F0E70122FBE70222F9E70322F7E70422F5E70522F3E7072218
:20080000F1E700229121E1E702221821DEE70622E9E70020DDE7036810B59B68044698470A
:2008200028B1A42104F10C00FFF77FFF10BD4FF0FF30FBE708B501210C30FFF776FF4011B1
:20084000431E5842584108BD10B50848FFF7E3FF431C044607D00548FFF7ECFF44EAC014A2
:20086000034BDC7210BD0024FAE700BF900300202401002008B501210C30FFF756FF40119C
:20088000831E5842584108BD38B500F10C05044648212846FFF749FF492184F828002846F5
:2008A000FFF743FF4A2184F829002846FFF73DFF94F8293094F828201B0284F82A0043EAA7
:2008C0000243C0B20021184338BD032108B50C30FFF72BFFC0B208BD272108B50C30FFF745
:2008E00024FFC0F3810008BD08B527210C30FFF71CFF431C0CBF002000F0030008BD08B5CB
:2009000062210C30FFF711FF431C0CBF002000F01F0008BD642108B50C30FFF706FF00F08B
:20092000030008BD08B524210C30FFF7FEFE431C1FBF00F0070000EB800000EB8000800035
:200940000CBF002000F6282008BD162108B50C30FFF7EBFE00F0070008BD08B5132972D89B
:20096000DFE801F00A18274547717171717171596567696B7375777982210C30FFF7D5FECB
:2009800000F01F0000EB800000EB8000800000F2DC5059E083210C30FFF7C7FE431C52D07F
:2009A00000F07F031846462B4FEA8303184414DC0BE084210C30FFF7B8FE00F07F03462B90
:2009C00018464FEA830204DC1044400000F5FA703AE0473B102B104402D88000C83804E0BF
:2009E00000EB80008000A0F5E15080B22CE08521D1E786210C30FFF798FE411C23D000F0FB
:200A00001F00192837D000EB800000EB8000800000F5AF6018E092210C30FFF786FE00F0C4
:200A20001F0000EB800000EB80008000CEE79321F2E79421F0E79521EEE796210C30FFF7FF
:200A400074FE421CEBD1002008BD9721F6E79921F4E79A21F2E76A210C30FFF766FE431CE7
:200A6000F1D000F0070000EB800000EB8000800000F62820E8E74FF49660E5E738B500F178
:200A80000C0500212846FFF750FE012104462846FFF74BFE240204F4F85400F01F0020437D
:200AA00038BD38B5036805469B68984708B9002038BD0C3534212846FFF737FE0446352117
:200AC0002846FFF732FE621CF1D0431CEFD0240204F4F854204380B2EAE773B586690446F4
:200AE0000D468DF8072036B10123007C0DF10702B04702B070BD4068B0B1217C01F096FE68
:200B00006068294603681B6898476068012203680DF107015B689847606802F00CF80038DD
:200B200018BF01204042E4E74FF0FF30E1E738B500F10C040D4620466921FFF7F6FD431CC1
:200B40000BD000F0C80242EA051242F005026921204602F0FD02FFF7C0FF38BD08B5FFF746
:200B6000A1FCBDE8084001210148FFF7E0BF00BF9003002010B51348FFF7FEFD00B311485C
:200B8000FFF749FE04462D2007F00AFB631E1F2B01460AD80120FFF78DFC0A48FFF74AFE61
:200BA00070B1BDE81040FFF7D9BFA4F12103202B01D80220EFE7423C222CEED80320EAE736
:200BC00010BD00BF90030020504BF0B45C6805680173002C00F09880002D00F09580AE7866
:200BE0004B4A013E28789278042E2ED8DFE806F025031D21290052067FD4002800F084802C
:200C000002290FD1A0F120035F2B0AD9A0F10803022B06D9D42804D000F14C03DBB2032B35
:200C20006ED801212346F0BC18475306E5D5A22064E05706E1D5A32060E05606DDD5A420D7
:200C40005CE05506D9D5A52058E0C12809D1012901BF93F8DB6083F8DA1086F0010683F882
:200C6000DB601206C9D593F8D72012B993F8D82032B1A0F14102192A01D96878BDE7012238
:200C800093F8DB501DB1A0F14105192D32D993F8D65015B993F8DD3023B301290BD100F0C5
:200CA000FD032C2B30D020282ED042282CD0492828D1D120B6E703299FD12C2804D16FF015
:200CC0000900F0BCFFF7A0BB2E2801D10A20F8E7202804D04228EAD1F0BCFFF74BBFF0BC44
:200CE000FFF7BCBB002A88D1A0F14103192B84D82030C0B2022995D193E7A120022991D174
:200D000002218FE700288DD1F0BC7047340100202401002038B5037B04460D46032B00F28F
:200D20009480DFE803F002304158002900F08D8003689A78474B1AB101211A4482F8D4103C
:200D400093F8DA1093F8D62089B1284693F8DC50002D4DD193F8D710002977D01AB140F214
:200D60000111A3F8DC10114600284AD04CE093F8D8000028EAD022B140F20111A3F8DA1034
:200D8000E3E71046E2E707F049FA6368C01AB0F5967F05D902212046BDE83840FFF714BF84
:200DA000002D52D10321F6E70029FBD007F036FA6368C01AB0F5967F47D907F02FFAA3681D
:200DC000C01A642841D902212046FFF7FDFE07F025FAA06039E003689A7822B11D4B1344DB
:200DE000002283F8D42000212160D4E7B1B90FE0A0B993F8D71021B9294693F8D80000280D
:200E0000F4D00120A3F8DA0041B993F8D71011B993F8D81011B10121A3F8DC101AB983F816
:200E2000DA2083F8DC201A6832B193F8DA0093F8DC1000B901B1904701212046FFF7C4FE7E
:200E400007F0ECF900236060A36038BD0028DCD10146D2E734010020FF222DE9F04F7D4B73
:200E600085B01A7007F0DAF97B4CD4F8D030C01A102840F2A8800026784B794DDFF8E491EF
:200E8000029303954FF0000BC846DA46029B012113F8017B3846029307F0EAF800213846DC
:200EA00007F044F9704B0193019B13F8010B0193FFF7F0FB012380F0010111F0FF0103FAF3
:200EC0000BF200F083809E4209D1BBF1040F01BF604B93F800C02CF0100C83F800C02AEA6C
:200EE000020A4FF0000C5C4B9A68424500F0AC800CF1010CBCF10A0F03F11403F4D140B9B6
:200F0000554A9168002972D001300A2802F11402F7D10BF1010BBBF1070F08F11808C3D123
:200F2000039B012103F801AB38460393013607F0FDF80021384607F09BF8082E09F10309AE
:200F4000A0D14FF0000B4FF00109DFF82081484E404FDFF804A118F8010BFFF79BFBBBF120
:200F6000070F80F00101C9B250D82B7800294AD003F07F032B70A4460023DCF80820B24253
:200F80005CD001330A2B0CF1140CF6D140B923469A68002A47D001300A2803F11403F7D1FD
:200FA0000BF1010B5FFA8BFBBBF10C0F06F1030605F10105CFD1FF22294B1A7207F02EF9A8
:200FC000254BC3F8D00005B0BDE8F08F012E09D1BBF1040F01BF1F4B93F800C04CF0100CA8
:200FE00083F800C04AEA02025FFA82FA79E7142358432218117501210830C2F808802044B7
:20100000FFF788FE85E763F07F03B3E7ABF10802D2B23B7809FA02F219B123EA02033B701E
:20102000A9E71343FBE7142301215843231808309E601A752044FFF76DFEB1E758B2142356
:2010400003FB00A00830F6E7142303FB0C400830D6E700BF040000203401002098970008F8
:201060005D020020E4960008A09700088C970008C0960008032910B5044602D9042904D090
:2010800010BDBDE81040FFF752BD0C3469212046FFF74BFB431CF3D000F0F90040F00102DF
:2010A00069212046FFF719FDEAE770B504460D461646FFF73AFB431C0CD0012303FA06F2C6
:2010C000024329462046D2B2FFF707FDB0FA80F0400970BD0020FCE708B5002210210C3099
:2010E000FFF7E3FF08BD000038B51348FFF793FB14280446114D18D82B6801332B60FFF76B
:20110000D5F9012C0BDC02210B48FFF710FD2CB92B68032B02D90848FFF7DEFF38BD0321B7
:20112000BDE838400448FFF702BD00242C60FFF7B9F92146F4E700BF90030020580200200B
:2011400008B500210348FFF7F2FCBDE80840FFF7CBBF00BF9003002008B5002268210C30FF
:20116000FFF7A3FF08BD08B5022230210C30FFF79CFF08BD08B5002230210C30FFF795FF58
:2011800008BD08B5032230210C30FFF78EFF08BD08B5012230210C30FFF787FF08BD08B568
:2011A000042230210C30FFF780FF08BD08B513292ED8DFE801F00A101214162D2D2D2D2D54
:2011C0002D181B1D1F212325272A002280210C30FFF76BFF08BD0122F8E70222F6E703226D
:2011E000F4E70422F2E700229021F0E70122FBE70222F9E70322F7E70422F5E70522F3E75C
:201200000722F1E700229121E1E702221821DEE70020DFE708B5002226210C30FFF745FF8D
:2012200008BD70B50446002500F10C06FF2248213046FFF752FCFF224921304684F8285019
:20124000FFF74BFCFF224A21304684F82950FFF744FC84F82A5070BD642238B5B1FBF2F5FB
:2012600002FB15139BB22BB11449154806F0FBFC002038BD40F62723994203D840F62822AE
:201280001049F2E740F6E442914201D90E49ECE700F10C0424212046FFF747FA431CE7D0F0
:2012A00000F0F800A5F11A02024324212046D2B2FFF713FCB0FA80F04009DAE77D8D0008E5
:2012C000F40600209F8D0008D78D000870B504460D461646FFF729FA431C0DD0012303FAC0
:2012E00006F220EA020229462046D2B2FFF7F5FBB0FA80F0400970BD0020FCE708B5012236
:2013000030210C30FFF7E2FF08BD08B5002230210C30FFF7DBFF08BD08B5042230210C3033
:20132000FFF7D4FF08BD08B5032230210C30FFF7CDFF08BD08B5022230210C30FFF7C6FF00
:2013400008BD08B5002268210C30FFF7BFFF08BD38B5036804465B6D0D46984728B12D49C0
:201360002D4806F080FC002038BD142DFBD801A353F825F0C9130008D7130008DB1300088D
:20138000DF130008E313000867130008671300086713000867130008671300086713000849
:2013A000E7130008ED130008F1130008F5130008F9130008FD13000801140008051400089D
:2013C0000B140008111400080022802104F10C00FFF77CFFC8E70122F7E70222F5E70322AF
:2013E000F3E70422F1E700229021EFE70122FBE70222F9E70322F7E70422F5E70522F3E75D
:201400000722F1E700229121E0E702221821DDE70622E9E70F8E0008F40600202DE9F84307
:201420000C460B462C49161E05462C4A2C4808BF0A462C4906F017FC14F0FF0710D005F1B6
:201440000C0740213846FFF770F9CEB344EA0002D2B23846402185F82B20FFF73EFB0746E3
:2014600014F47F4F13D005F10C08412140464FEA1429FFF75AF936B349EA00095FFA89F209
:201480004121404685F82C20FFF727FB074314F47F0F10D005F10C0842214046240CFFF7AA
:2014A00044F9A6B10443E2B24221404685F82D20FFF713FB0743B7FA87F04009BDE8F8832B
:2014C00020EA0402C4E720EA0902D2B2D8E720EA0402D2B2E8E700BF608E0008598E0008F2
:2014E000F4060020688E000808B511460022FFF795FF08BD08B511460122FFF78FFF08BDCF
:2015000038B500F10C040D4620462721FFF70DF9431C0CD000F0F30242EA8502272120465F
:20152000D2B2FFF7DAFAB0FA80F0400938BD0020FCE738B500F10C040D4620462721FFF71D
:20154000F4F8431C0BD000F0FC0045EA000227212046FFF7C2FAB0FA80F0400938BD002070
:20156000FCE7102938B50D4601D9002038BD00F10C0462212046FFF7D8F8431CF5D000F05C
:20158000E00045EA000262212046FFF7A6FAB0FA80F04009EAE7052938B50D4601D900201F
:2015A00038BD00F10C0464212046FFF7BEF8431CF5D000F0FC0045EA000264212046FFF77C
:2015C0008CFAB0FA80F04009EAE738B500F10C050C4628461621FFF7A8F8431C0CD000F0AA
:2015E000F80004F00702024316212846FFF775FAB0FA80F0400938BD0020FCE738B500F16E
:201600000C050C4628468321FFF78FF8431C11D0A4F5FA73B3F52F7F00F0800018D80A22B0
:20162000B4FBF2F302FB1344A4B22CB11049114806F019FB002038BDA3F13202024383210D
:201640002846D2B2FFF749FAB0FA80F04009F2E7A4F2C443B3F5A07FECD81422B4FBF2F331
:2016600002FB1344A4B2002CE0D103F10A02E5E7788E0008F406002038B500F10C050C46AE
:2016800028468421FFF751F8431C12D0A4F5FA739AB2B2F52F7F00F0800018D80A22B4FBD5
:2016A000F2F102FB114189B229B11949194806F0DAFA002038BDB3FBF2F202438421284657
:2016C000D2B2FFF70AFAB0FA80F04009F2E7A4F2C443B3F5A07F0AD81422B4FBF2F302FB43
:2016E0001344A4B2002CE0D103F10A02E5E7A4F5C863B3F5E16FDCD86422B4FBF2F302FB0D
:201700001344A4B2002CD0D103F14802D5E700BF9A8E0008F406002038B500F10C050C460B
:2017200028468521FFF701F8431C11D0A4F5FA73B3F52F7F00F0800018D80A22B4FBF2F3EA
:2017400002FB1344A4B22CB11049114806F08BFA002038BDA3F13202024385212846D2B21B
:20176000FFF7BBF9B0FA80F04009F2E7A4F2C443B3F51B7FECD81422B4FBF2F302FB1344C2
:20178000A4B2002CE0D103F10A02E5E79A8E0008F4060020642238B5B1FBF2F302FB1313D9
:2017A0009BB20C4623B11E491E4806F05CFA0DE0B1F5966F12D0B1F5AF6F09D24FF4AF632F
:2017C0004FF496621849174806F04DFA002038BD40F67462914201D91449E5E700F10C05D8
:2017E00086212846FEF7A1FF431CEFD0B4F5966F1EBF6423A4F5AF64B4FBF3F400F0E002FB
:2018000018BF22434FF0860128460CBF42F01902D2B2FFF762F9B0FA80F04009D7E700BF8B
:201820007D8D0008F4060020BB8E0008E78E000870B56426B1FBF6F306FB13139BB20C46A4
:2018400033B132461549164806F00DFA002070BDB1F5FA7F03D24FF4FA721249F3E740F618
:20186000AC52914201D91049EDE700F10C0596212846FEF75AFF431CE8D0A4F5FA74B4FB4E
:20188000F6F400F0E00044EA000296212846D2B2FFF723F9B0FA80F04009D8E77D8D00086F
:2018A000F40600200D8F00083D8F000870B56426B1FBF6F306FB13139BB20C4633B1324630
:2018C0001449154806F0CFF9002070BDB1F5FA7F03D24FF4FA721149F3E740F648529142C9
:2018E00001D90F49EDE700F10C0599212846FEF71CFFA4F5FA74B4FBF6F400F0E0002043D5
:20190000C2B299212846FFF7E8F8B0FA80F04009DBE700BF7D8D0008F40600206D8F000841
:201920009D8F0008642238B5B1FBF2F502FB15139BB22BB11349144806F095F9002038BDCE
:2019400040F62723994203D840F628220F49F2E740F6E4429142F9D800F10C046A212046AE
:20196000FEF7E3FE431CE9D000F0F800A5F11A0202436A212046D2B2FFF7AFF8B0FA80F06E
:201980004009DCE7CD8F0008F406002005900008036870B55B6D05460E461446984728B117
:2019A0009B499C4806F05FF9002070BD142EFBD801A353F826F000BF0D1A00085F1A00083B
:2019C000691A0008731A00087D1A0008A9190008A9190008A9190008A9190008A919000856
:2019E000A9190008871A0008D11A0008191B0008631B0008AD1B0008AD1B0008B71B000845
:201A0000B71B0008C11B0008CB1B00086421B4FBF1F301FB13439BB213B164227E4906E06C
:201A200040F2DB539C4206D840F2DC527B49794806F019F9B8E740F64852944201D97849BD
:201A4000F5E7A4F2DC52B2FBF1F28221D2B205F10C00FFF742F8B0FA80F04009A5E72146A7
:201A60002846FFF7CBFDA0E721462846FFF704FE9BE721462846FFF74FFE96E721462846FA
:201A8000FFF788FE91E76426B4FBF6F306FB13439BB2002BC1D1B4F5FA7F03D24FF4FA7229
:201AA0006049C4E740F6AC52944201D95E49BEE70C3592212846FEF738FEA4F5FA74B4FB5F
:201AC000F6F4922100F0E0022243D2B22846C0E76426B4FBF6F306FB13439BB2002B9CD13B
:201AE000B4F5FA7F03D24FF4FA7250499FE740F6AC52944201D94E4999E70C3593212846C3
:201B0000FEF713FEA4F5FA74B4FBF6F400F0E00222439321D2B2D9E76426B4FBF6F306FBCD
:201B200013439BB2002B7FF478AFB4F5FA7F03D24FF4FA723F497AE740F6AC52944201D9CA
:201B40003D4974E70C3594212846FEF7EEFDA4F5FA74B4FBF6F400F0E00222439421D2B250
:201B6000B4E76426B4FBF6F306FB13439BB2002B7FF453AFB4F5FA7F03D24FF4FA722F4946
:201B800055E740F6AC52944201D92D494FE70C3595212846FEF7C9FDA4F5FA74B4FBF6F4B9
:201BA00000F0E00222439521D2B28FE721462846FFF73EFEF9E621462846FFF777FEF4E63E
:201BC00021462846FFF7AEFEEFE63222B4FBF2F602FB16439BB2002B7FF420AFB4F5FA7F9C
:201BE00003D24FF4FA72174921E7B4F5AF6F03D94FF4AF6214491AE70C3598212846FEF747
:201C000094FD0A3E00F0E00232439821D2B25DE758900008F40600207D8D00089E900008D1
:201C2000C5900008EC9000081C9100084C9100087C910008AC910008DC9100080C920008B4
:201C40003C9200086C9200089D9200082DE9F043012185B00D2006F00BFA00210D2006F065
:201C600065FA0A20FEF71EFD06F0DAFA06224FF4E131774805F054FF764B77495A6E002410
:201C8000C1F884201B6E7448C1F8883000231F211A4601F01AF842F210716F4800F0ACFD66
:201CA0006E4B694600936E4B6B4803936D4B0194029300F0C3FD6846FEF7EDFA6A4F6B4B9C
:201CC0006B4E6946644801946A4C00930397029600F0E4FD6846FEF7DEFA94F80C80B8F1D3
:201CE000000F00F092802046FEF726FB002840F0A3806149564805F0A3FF00212C2006F09A
:201D0000B7F901212D2006F0B3F900212D2006F00DFA01210E2006F0ABF901210E2006F067
:201D200005FA42F2107006F02FF96421082006F031F9FEF781FC514B514A6FF0DE005A6065
:201D4000FEF762FB01210D2006F0F0F94FF42F614848FFF781FA4748FFF7D0FA4548FFF75D
:201D6000FBF94448FFF7FFF94248FFF703FA4148FFF707FA04213F48FFF77CF90221292075
:201D800006F076F9002301933E4B6946032229200093CDE9026706F009F86846FEF77BFAC0
:201DA0004FF0FF3200233348FFF79EFB3148FFF738FA354A00232F48FFF79CFB1A21334889
:201DC000FEF7B3FC421C05D000F00F021A212F48FEF783FE1A212D48FEF7A7FC431C07D085
:201DE00000F0F00040F001021A212848FEF775FE0022274B1A600122264B1A70FEF724FD7B
:201E000005B0BDE8F043FFF76FB901231B214FF01A09214D23732846C4E905192561FEF79D
:201E200067FA49462846FEF73FFA4146284600F047FF3423237756E70122184B0D481A7058
:201E4000FEF743FD16490246014805F00CFF54E774020020289C0008A804002001250008C6
:201E600091020008710200086D020008652600084D02000890030020CE920008340100207B
:201E8000950500080D02000800FC18009C0300208C030020C1030020C4030020C203002057
:201EA000E392000870B516460546FEF73EFC044631462846FEF739FC621C07D0431C05D0C8
:201EC000240204F47C54204380B270BD0020FCE7036810B5DB680446984728B13922382126
:201EE00004F10C00FFF7DEFF10BD08B53B223A210C30FFF7D7FF08BD10B55A495A4805F000
:201F000085FE5A48FEF796FC594C5A49002818BF2146554805F094FE5749534805F076FE9F
:201F20005248FEF7A7FC5349002818BF21464E4805F086FE51494C4805F068FE012150481B
:201F4000FEF7F3FB4B4B400914BF19462146464805F076FE4B49444805F058FE4348FEF744
:201F600012FC4449002818BF21463F4805F068FE45493D4805F04AFE052200214048FEF769
:201F8000E4FB3C49002818BF2146374805F058FE3E49354805F03AFE01213948FEF7C5FB24
:201FA000431C5DD000F00700052808D8DFE800F003505254565836492B4805F041FE35498F
:201FC000294805F023FE2948FEF76BFD0A220146254805F094FE3049234805F031FE2F49C5
:201FE000214805F013FE2148FFF772FF0A2201461D4805F084FE28491B4805F021FE2849FA
:20200000194805F003FE1948FFF76FFF0A220146154805F074FE2049134805F011FE13484A
:20202000FEF7AAFB78B11F490F4805F0EFFD0F48FEF7F1FB0A2201460B4805F060FE1A4989
:20204000094805F0FDFDBDE81040074805F0E6BD1649B1E71649AFE71649ADE71649ABE794
:202060001649A9E7F69200087402002090030020EF920008F3920008029300080F9300083B
:202080009C0300201A93000824930008309300084293000891930008D48D0008A193000894
:2020A000B1930008C3930008D69300084D93000858930008689300087993000885930008F3
:2020C00073B5074B1B784BB1012B0DD04FF47A70584306F0A5F80348FEF7FEFF02B070BD77
:2020E000C20300209003002006F098F8A64C2368C01A44F62063984212D906F08FF82060EC
:20210000A248FEF788FB0446601C00F0A6819F48FEF790FB44EAC014FEF7E6FF9C4BDC7208
:202120009C4B1A78002AD9D00022984C1A702046FEF7AAFB05469849984805F067FD10222C
:202140002946964805F0DDFD9549944805F05EFD02222946914805F0E1FD94F92B30002B07
:2021600007DA94F92830002B03DA8E498B4805F067FD94F82B3059060AD594F828305A0625
:2021800006D58949854805F05BFD8048FEF7A4FF94F82B309B0607D594F828309E0603D554
:2021A00082497E4805F04CFD94F82B301D0707D594F82830180703D57D49784805F040FDD6
:2021C00094F82B30990707D594F828309A0703D57849724805F034FD94F82B30DB0707D5F9
:2021E00094F82830DE0703D573496C4805F028FD6648FDF7B4FF18B17049684805F020FD1B
:202200006248FDF7B5FF28B16D49644805F018FDFEF796FF5D48FDF7B6FF70B15B48FEF796
:20222000FAFA451C08BF0020594B18BF40F08000D8726449594805F003FD5448FDF7AEFF6D
:2022400040B10022524B60495448DA7205F0F8FCFEF776FF4D48FDF7ACFF38B35B494F4890
:2022600005F0EEFC01219120FEF794F958494B4805F0CCFC04230025194656480DEB0302F3
:202280000195FEF71FFA01AE0A2216F8011B434805F042FD01355049404805F0B7FC042DA6
:2022A000F2D13E4805F0BAFCFFF726FE3748FDF78BFF90B14949394805F0C2FC00210D20BE
:2022C00005F034FF00210E2005F030FF2F480421FEF7D0FE2D48FEF7FFFE94F82C30980716
:2022E00007D594F82930990703D53D492B4805F0A7FC94F82C30DA0707D594F82930DB07A8
:2023000003D53849254805F09BFC94F82D305E0607D594F82A305D0603D533491F4805F049
:202320008FFC94F82D30980607D594F82A30990603D52E49194805F083FC1448FDF74FFF68
:2023400080B11248FEF767FA421C08BF0020104B18BF40F08000D8722549104805F070FC04
:20236000FEF7EEFE0948FDF745FF00284DD00748FEF751FA431C08BF0020054B18BF40F082
:202380008000D8721B4937E08C0300209003002024010020C3030020D89300087402002062
:2023A000E7930008ED9300080194000815940008229400083D940008569400087094000830
:2023C0007D9400088A94000896940008A2940008B49400089C030020CB940008CD9400086F
:2023E000DE940008EE940008FE940008129500082995000839950008194805F021FC194820
:20240000FEF7BAF908B1FEF7A9FB94F82D305E0707D594F82A305D0703D51349104805F0CD
:202420000FFC94F82D30980707D594F82A30990703D50E490A4805F003FC94F82D30DA0768
:2024400007D594F82A30DB0703D50949044805F0F7FB0448FEF7E5FE40E600245EE600BF0A
:2024600074020020900300204A950008629500087695000808B5FFF723FEFEF7EDFCFDF774
:2024800095FFBDE808400A2005F0CABE07B51A221B210F4800F022F9002205210D4B0E4888
:2024A000C3E908221A739A600C4A19711A600C4A17211A611622C3E9051234221A77332324
:2024C00009220A21009305F0D9F903B05DF804FBC40300209003002074020020C8950008B0
:2024E000A804002008B50448FDF796FEBDE80840024800F06DB900BF90030020C4030020D9
:2025000037B54C4800F0C4F800282CDD0024494800F0BEF8B0B9484C9DF8003020706070E1
:202520000220464903F07F03043B9DF9002008700A2B18D8DFE803F03819171766112633DA
:20254000465459003B4800F0A7F804F108036B4403F8080C84F00104D9E7FEF749F8C0F396
:2025600007232370607003B030BD002A344D04DA9DF801306B71FDF737FF052323706B793A
:202580006370F0E7002A2E4D05DA9DF801300020AB72FDF74BFF0A232370AB7AF0E70B23E2
:2025A0002370274BDB7AEBE7264B93F8DD2093F8DB305B0143EA8213234A92F83E20134397
:2025C0002370D0E70C232370204B21481A68C4F801205A681B7A426003720A230B70C2E7FD
:2025E0000D2323701B4B1B78CAE7002A06DA9DF80120194B052A98BF06221A700E2323704E
:202600000123BDE7002ABBBF4FF47A709DF801304FF47A70584305F003FEBFF34F8F0F49B5
:202620000F4BCA6802F4E0621343CB60BFF34F8F00BFFDE7A8040020670200206602002045
:202640002401002034010020140200205D0200206802002004000020C203002000ED00E0CB
:202660000400FA05064B1A78531E092B03D80549054800F0B5B90021034800F090B900BF97
:202680006602002067020020A804002000207047028BC08A101A70470346C28A018B9142DA
:2026A00081BF0169885C0132DA8298BF4FF0FF307047028BC38A9A4286BF0269D05C4FF0B0
:2026C000FF307047806DD0F8DC302BB10023D43020F8B23CC36818477047000070B54FF4A1
:2026E0007A730E460021C0E90113034615462B4A044643F8C42BC0F8C4109C22C3E9011126
:20270000C0E93411C0E93611C0F8E010283005F017FFF3B2322B19D8214A06F4E06652F8E8
:2027200023301E43EBB2322BC4F8846022D81C4A05F4E06552F823301D4300232046C4F86B
:202740008850E36123842361A38270BD06F0C002C02A0CD1CF2B0AD8124B06F03F0253F8A6
:2027600022200F4B06F4E06653F82230D9E74FF0FF36D7E705F0C002C02A0CD1CF2B0AD894
:20278000084B05F03F0253F82220054B05F4E06553F82230D0E74FF0FF35CEE7B0970008CA
:2027A000289C0008E89B000838B50446283000F055FBE06918B105F05BFD0023E361002508
:2027C0002069258410B105F053FD2561A58238BD38B505460446074B45F8D43BFFF7E4FF26
:2027E0002846FDF758FD04F1C400FDF754FD204638BD00BFB097000838B5044600F1280566
:20280000284600F069FB94F8BE304BB92846054900F062FC2846BDE83840034900F055BC96
:2028200038BD00BFC5260008212900080123994080F8243000238176438470470023F0B576
:2028400087B002AC02930593C4E901338B6805460E460BB3022220469847D6E9023794E858
:202860000300CDE9000105F1C40292E8030084E80300DDE9000182E80300D5F8CC20C5F84C
:20288000CC30D5F8D0302046C5F8D07004920593FDF701FD07B0F0BD1F46E0E70023F0B594
:2028A00087B002AC02930593C4E901338B6805460E460BB3022220469847D6E9023794E8F8
:2028C0000300CDE9000105F1D40292E8030084E80300DDE9000182E80300D5F8DC20C5F8CC
:2028E000DC30D5F8E0302046C5F8E07004920593FDF7D1FC07B0F0BD1F46E0E738B5838A03
:2029000005468B420C4609D2202938BF20240069214605F063FD10B12861AC8238BDFEE777
:2029200073B5846D0546D4F8CC30866EE3B1E28A238B9A4218D331462046FFF7DFFF3246D9
:20294000206905F1740105F04BFE0023E382D4F8CC30268301960BB906F0E8F9D4F8D0304E
:2029600001A904F1C400984702B070BDB1F5806F70B505460C4610D8038C99420AD9202961
:202980000E4638BF2026C069314605F027FD18B1E8612E84204670BDFEE70024FAE713B5E4
:2029A00090F8243004468DF807107BB1418C0131FFF7DCFF40B10120638C9DF80710E26961
:2029C000D154638C0133638402B010BD01220DF10701283000F0A8FAB0FA80F04009F3E7F9
:2029E00070B590F8243004460E46154693B1418C1144FFF7BBFF10B90025284670BD638C4F
:202A0000E0692A461844314605F0EAFD638C2B446384F2E792B2283000F086FA0028EBD140
:202A2000EBE70346006918B100219A8A05F088BD70470346C06918B100211A8C05F080BDDF
:202A4000704738B50446D1B94FF42A03A36594F8BE30012B16D1638CE269A17E04F1280083
:202A600000F0E2FA042828BF0420C5B22046FFF7E0FF0023638484F82430284638BD4FF025
:202A80002A43E3E70425F8E72DE9F04790F8BEA00446BAF1010F0F46154698469DF820601C
:202AA0009DF8249039D111467F00FFF727FFFFB27EB10023032E28BF032684F824A0A77630
:202AC0006384013EF6B2FF2E1BD100212046FFF7B8FFB9F1000F1DD14FF42A03A36539463D
:202AE0002B46226904F1280000F038FA002398422E461CBF1D462E462846E3822683BDE857
:202B0000F0872368F10028FA01F120461B68C9B29847D6E74FF02A43E0E70020EFE707B589
:202B2000019300230093FFF7AFFF03B05DF804FB0123FFF7F4BF0121FFF783BF38B5002567
:202B40000446C5820583FFF76CFF20466584FFF770FF38BDF8B50446D0F8840005F0C2F95F
:202B6000002105F085FAD4F88420C2F30313042B48D8284D284E55F8233002F00F029B68A5
:202B800056F82220DB4303EA12239BB2002B3FD0D4F8880005F0A6F9012105F069FA1F4B12
:202BA000D4F888001B681E4CC0F30311B3FBF4F30A24042904FB03F300F00F0225D81427EF
:202BC00056F82220174CC2F30F2255F821C0CCF81420D4F804E06668A6EB0E06B342FADC08
:202BE000CCF81020D4F804C06668A6EB0C06B342FADC013FE9D105F075F93946BDE8F8405C
:202C000005F036BA00239B68FFDE00235B61FBE7F8BD00BF0C000020F49700082800002090
:202C200040420F00001000E02DE9F04100260446C68206831F460D469046FFF7F2FE2046B1
:202C40006684A676FFF7F5FED4F8DC30C4F8804033B104F1D401032208469847C4E93766E7
:202C6000002384F824306B0084F825306B1E5D425D41204684F8BE5084F8BF8084F8C07008
:202C800004F12805FFF766FF284694F82520094900F02CF894F8BE304BB92846064900F0E7
:202CA0001BFA2846BDE8F041044900F00EBABDE8F08100BFA0860100C52600082129000875
:202CC0000A4600230121FFF7AFBFC9B2FFF7ACBF162217210148FFF701BD00BFA804002027
:202CE0000148FFF775BD00BFA8040020F7B50D4617460446002800F09F805049C06D04F041
:202D00008DF84F490646206E04F088F80146002E00F09280002800F08F80304604F0A5F8A3
:202D20002060002800F08880464B261D984260D103F5DE33DA6942F40012DA61DA6902F40C
:202D400000120092009A1A6942F400121A611A6922F400121A6142F21F03A4F864303A4BBE
:202D60001E603749206E04F041F83449E06D04F03DF8364B21689D4258D9354B9D4203D952
:202D8000344B9D4288BF00234FF480420025C4E901134FF48043C4E9053594F8973002211D
:202DA0005B1B18BF01239B01236294F89830C4E903275B1B18BF0123DB0163622A4694F947
:202DC0006400E56184F8415000F09EFA94F9640000F0CAFA2A46022194F9650000F094FA0C
:202DE00094F9650000F0C0FA304600F0AFFCF8B1FEE7194B9842B4D103F5DC33DA6942F455
:202E00008002DA61DA6902F480020192019A1A6942F480021A611A6922F480021A6142F28C
:202E20002123A4F86430084B5E609AE70022ADE70223A06684F8953003B0F0BDB89B0008AF
:202E4000889B0008005400408C050020A0860100801A060040420F000058004010B5044603
:202E600090F9640000F08EFA94F9650000F08AFA201D00F014FD0321206E03F0F7FE03218B
:202E8000E06D03F0F3FE2368104A93420DD1104B1A6942F400121A611A6922F400121A61A2
:202EA000DA6922F40012DA6110BD0A4A9342FBD1074B1A6942F480021A611A6922F4800287
:202EC0001A61DA6922F48002EDE700BF005400400010024000580040104B10B59942044646
:202EE00006D90F4B994203D90E4B994288BF00236068026822F001020260A360074B201D09
:202F0000994294BF002101218903E16000F01EFC6268136843F00103136010BDA086010086
:202F2000801A060040420F00202A30B514D800239CB2A24207D890F894301344DBB280F869
:202F40009430002030BD90F89440CD5C1C44044484F874500133EBE70120F3E72DE9F347E2
:202F600005460F469046994600F0B6F900240646D5F830A004354B46424639462846CDF84C
:202F800000A000F0B9FD022806D100F0A5F9841B642CF0D906201FE008BB00F09DF90646AA
:202FA000284601F01FFD202809D0632C07D800F093F9841B284601F018FD0028F0D0284622
:202FC00001F013FD632C0CD882060AD443070AD4003818BF0120800002B0BDE8F08704204D
:202FE000FAE70520F8E70320F6E710B564230446043000F06DFC022810D0032806D090B17D
:2030000094F84130202B18BF042004E094F84130202B18BF052008BF022004E094F841307B
:20302000202B18BF062010BD2DE9F34704460E4691461F4600F050F980463FB901223146C0
:20304000204602B0BDE8F047FFF7CFBF0025D4F830A004343B464A4631462046CDF800A0AC
:2030600000F0E2FC022807D100F036F9A0EB0805642DEFD906201FE008BB00F02DF9064626
:20308000204601F0AFFC202809D0632D07D800F023F9851B204601F0A8FC0028F0D02046A9
:2030A00001F0A3FC632D0CD882060AD443070AD4003818BF0120800002B0BDE8F0870420DC
:2030C000FAE70520F8E70320F6E720B119B1C166043000F00DBE704720B119B1016704306C
:2030E00000F006BE704770B590F891300446012B0D46A0F1040609D1436E3BB1836E3046B5
:203100009847022384F89130002363668DB9E36E84F891501BB1304684F8905098472046AB
:2031200094F8902004F170012023BDE8704000F069BD00230122636684F89120616E2046CE
:20314000743131440423BDE8704000F096BD10B590F891300446012B04D1436E13B1836ED7
:2031600004389847022384F89130002320466366BDE8104000F0BCBD436E1F2BDEBF436ED9
:203180000133436690F89130012BDAB205D1416E04237031014400F070BD7047002380F850
:2031A0009030704790F892300BB900F0A1BD7047014B186800F01CBF8C050020014B186871
:2031C00001F070BB8C050020014B586800F010BF8C050020014B586801F064BB8C050020D9
:2031E0000379012B07D10A2919D840F2C740C84000F001007047022B0BD1022903D8081E0D
:2032000018BF01207047063903298CBF002001207047042B03D1142901D80248E7E7002000
:20322000704700BF1FF81900012303FA01F183680B4383607047012303FA01F1836823EAF7
:203240000103836070478068C84000F0010070477047000038B50E4B05461A784FF47A732E
:20326000B3FBF2F30B4A1068B0FBF3F000F09CF8044658B90F2D09D8024629464FF0FF303F
:2032800000F042F82046044B1D6038BD0120FCE7050000202800002008000020074A08B536
:2032A0001368032043F01003136000F01BF80020FFF7D0FFFFF7CCFF002008BD00200240C7
:2032C000034A044B11681B780B441360704700BF9405002005000020014B1868704700BFEE
:2032E0009405002007490302CA6803F4E06322F4E0621204120C134343F0BF6343F40033B3
:20330000CB60704700ED00E0154B30B5DC68C4F30224C4F10703251D042B28BF0423062D27
:203320004FF0FF3594BF0024033C05FA03F321EA0303A54022EA0502A340002843EA020329
:20334000ACBF00F16040074A4FEA0313DBB2ABBF00F5614000F00F0080F80033135430BD46
:2033600000ED00E014ED00E0002807DB01234109034A00F01F00834042F82130704700BF07
:2033800000E100E000280CDB01220649430900F01F008240203341F82320BFF34F8FBFF3BD
:2033A0006F8F704700E100E00138B0F1807F0BD24FF0E023F021054A586182F823100020B9
:2033C000072298611A6170470120704700ED00E0002808DB01224309034900F01F0082405D
:2033E000603341F82320704700E100E0704708B5FFF7FCFF08BD704710B5044650B1437999
:2034000003F0FF0213B90271FFF7F5FF01230020637110BD0120FCE790F821200346022A68
:2034200006D0042282630120002283F8202070470268C06B116821F00E011160116821F0CD
:203440000101116001211A6C01FA02F24260002083F82110E8E7000008B590F82130022B62
:2034600003D004238363012008BD03681A6822F00E021A601A6822F001021A60174A9342B6
:203480001FD0143293421ED0143293421DD0143293421DD0143293421DD01432934214BF2E
:2034A0004FF080734FF480130D4A5360012380F82130002380F82030436B03B198470020C1
:2034C000D2E70123F0E71023EEE74FF48073EBE74FF48053E8E74FF48033E5E70800024037
:2034E0000000024090F82100704700002DE9F74F00244FF00F0E2646DFF884C1614B00F129
:2035000004080A6832FA06F502D103B0BDE8F08F012505FA06F702EA070537EA020276D1D6
:203520004A68032A07D8013A022A00F28380DFE802F091969C00122A00F0948069D8112A39
:2035400000F08A80FF2D94BF8146C1464FEA8602D9F8007088BF203A0EFA02FA27EA0A075B
:2035600004FA02F21743C9F80070D1F8049019F0805F4CD0DCF8182026F0030742F001020C
:20358000CCF81820DCF8182007F1804702F00102019207F5803706F0030A019A4FEA8A0ABE
:2035A000BA680EFA0AFB22EA0B0B374A904260D002F5806290425ED002F5806290425CD087
:2035C00002F58062904214BF0422032202FA0AF242EA0B02BA609A6819F4801F14BF2A43E9
:2035E000AA439A60DA6819F4001F14BF2A43AA43DA605A6819F4003F14BF2A43AA435A601A
:203600001A6819F4803F14BF2A43AA431A60013677E7DFF878904A450CD014D8A9F58019B3
:203620004A4507D009F570294A4503D0A9F580194A4587D18A68D2B1012A4FF008040CBF57
:20364000076147617EE7DFF848904A45F2D009F58039EDE7CC6875E7CC68043472E7CC68E1
:2036600008346FE7CC680C346CE700246AE7042468E70022AAE70122A8E70222A6E700BF30
:203680000010024000040140000801400000221000003110044A08B55169014202D050614C
:2036A00003F0ECF808BD00BF000401402DE9F84606460F4691461D464FEA114A3368BAF161
:2036C000010F39D15C6927EA0404A4B2B4FA84F46409A14501D0002024E06A1CEFD0FFF7F3
:2036E000FBFD089BC01AA84201D8002DE6D1BAF1010F336818D15B6927EA03039BB2B3FA9A
:2037000083F35B099945D9D1002320220120336386F83D2086F83E30326C86F83C3042F0AA
:2037200020023264BDE8F8869B69DB43C3F3400383F00103DBB2E5E79C69E443C4F340049C
:2037400084F00104E4B2C4E77047000070B5044608B9012070BD90F83D3003F0FF021BB9BD
:2037600080F83C20FFF7F0FF242384F83D3023681A6822F001021A601A6842F400421A6050
:203780001A6822F400421A6001F090FB3F4B65689D4294BF3E4B3F4B98428CBF0023012351
:2037A000002BD6D1394E3C4BB542B0FBF3F388BF4FF496762268516821F03F0141EA030148
:2037C00082BF73434FF47A76B3FBF6F35160116A013321F03F010B431362D169431E2B48A6
:2037E00021F44F41854221F0FF0132D86D00B3FBF5F340F6FC700133034242D0C3F30B034E
:203800001943D1611168D4E9073021F0C00103430B4313609168D4E9030321F40341034379
:2038200021F0FF010B439360D168D4E9053021F0FF0103430B43D3601368002043F0010361
:2038400013602023206484F83D30206384F83E0080E7A06850B905EB4505B3FBF5F301338C
:20386000C3F30B037BB143F40043C9E719206843B3FBF0F30133C3F30B0323B143F4404333
:20388000BEE70423BCE70123BAE700BFA08601007F841E00FF083D0040420F00704710B59C
:2038A000044698B12423026880F83D30136823F001031360FFF7F2FF0020206484F83C0097
:2038C00084F83D00206384F83E0010BD0120FCE72DE9FF4704461F4689469246FFF7FCFC81
:2038E00094F83D300546202B03D0022004B0BDE8F08700901923012220464949FFF7D6FEC3
:203900000028F2D194F83C30012BEED0012384F83C30236800261A6809F0FE09D2075EBFA5
:203920001A6842F001021A601A6822F400621A60242384F83D303B4B2664E36222684FF094
:2039400001111368204643F4807313603B4600220095FFF7ABFE236838B11B680320DB0506
:2039600044BF4FF400732364C0E7C3F81090FFF7B3FC4FF0A0080546226853695269C3F377
:203980004003C2F3802294F83D10A02901D013431DD04FF02008206884F83D80436913F000
:2039A000020F036843F40073036025D000230393436901220393836919490393039B204683
:2039C00019230095FFF772FE88B101208EE7FFF783FC401BB84200D80FB984F83D802268B4
:2039E00053695269C3F34003C2F38022CBE784F83D8084F83C0079E76FF4806301224361F0
:203A00000749192320460095FFF750FE0028DCD10136564592D384F83D8084F83C00D4E723
:203A2000020010000000FFFFF7B5002504460095019594F83D500898202D02D0022003B083
:203A4000F0BD25682E68B60503D4082801D001281BD146F2A817274E3668B6FBF7F6192706
:203A60007E430196019E013E0196019E56B92023266384F83D3084F83E60236C43F0200317
:203A80002364DBE7AE69B707ECD494F83C60012ED4D02E68F6075EBF2E6846F001062E603C
:203AA0002E6826F400662E60212684F83D60102684F83E60002626646385638DE062616423
:203AC0002385236B62620093009B112B05D1B0F52A0F02D0B0F12A4F03D12B6843F4807351
:203AE0002B60002084F83C006B6843F4E0636B60A5E700BF28000020F7B500250446009508
:203B0000019594F83D500898202D02D0022003B0F0BD25682E68B60503D4082801D00128D6
:203B20001BD146F2A817364E3668B6FBF7F619277E430196019E013E0196019E56B92023E4
:203B4000266384F83D3084F83E60236C43F020032364DBE7AE69B707ECD494F83C60012EBF
:203B6000D4D0012684F83C602E68F6075EBF2E6846F001062E602E6826F400662E60222665
:203B800084F83D60102684F83E60002626646385638DE06261642385236B62620093638DB0
:203BA0009BB2022B24D1202801D0102820D1009B122B2B681DD14FF4407223F480632B6081
:203BC0002B6843F400632B60009B122B05D1B0F52A0F02D0B0F12A4F03D12B6843F4807324
:203BE0002B60002084F83C006B6813436B608EE72B6843F480634FF4E0622B60E4E700BFB2
:203C00002800002037B5044690F83D0000F02800282830D100292CD0002A2AD094F83C00E7
:203C2000012828D025682868C0075EBF286840F001002860286820F400602860292084F8C8
:203C40003D00202084F83E00002020646285628DE36201906B6961620193AB6984F83C00E6
:203C60000193019B6B68228543F4E0636B6003B030BD0120FBE70220F9E737B5044690F8F2
:203C80003D0000F02800282830D100292CD0002A2AD094F83C00012828D025682868C00768
:203CA0005EBF286840F001002860286820F4006028602A2084F83D00202084F83E000020F5
:203CC00020646285628DE36201906B6961620193AB6984F83C000193019B6B68228543F4DC
:203CE000E0636B6003B030BD0120FBE70220F9E790F83D30202B14D1282380F83D30036851
:203D000000201A68D2075EBF1A6842F001021A601A6842F480621A605A6842F440725A6062
:203D200070470220704770477047704790F83D2008B5036DD2B283B9C36C0268012B836C48
:203D400005D1DBB21361036D0233036508BDC3F307231361036D0133F7E7036D012B03D174
:203D6000836C0268DBB2F4E7036D022B2FD1222A05D10268136843F480731360EAE7438DA0
:203D80009BB263B1212A0AD1436A026813F8011B11614362438D013B9BB24385D6E7438D99
:203DA0009BB2002BD2D1212AD0D10268516821F4E0615160116841F400711160202203639A
:203DC00080F83D2080F83E30FFF7AFFFBEE703685A69120644BF00221A61B7E770477047ED
:203DE000002337B546F2A81101932C4B406A1B6890F83D20B3FBF1F323214B430193036843
:203E0000D2B2019941BB016C41F020010164446B0CB10021A162816B09B100258D621D6895
:203E200025F480651D600025458504B1656301B14D63196821F00101196090F83D106029CE
:203E400011D1202380F83D30002380F83E300364FFF7C5FF03B030BD0199013901911968A7
:203E60008905CED4D3E702F02802282A0ED1196841F001011960196841F4806119600023AB
:203E8000036380F83D20FFF78DF9E3E7202380F83D30002380F83E30F5E700BF280000208D
:203EA00010B590F83D2090F83E300446102BD9B2D2B2036801D0402913D1222A11D1196896
:203EC00021F400611960596811F4006106D1602A1EBF202284F83D2084F83E100022226302
:203EE00007E002F028012829EDD10022226384F83D105A6812F400624FD05A68606B22F455
:203F000000625A6090F82130012B374B2BD04363FFF7A2FA50B12268606B136823F00103E3
:203F20001360202384F83D30436B9847236C19071FBF2268536823F4E063536094F83D307D
:203F4000226CDBB252070DD5282B0BD1274B2022E36200232046236384F83D2084F83E3011
:203F6000FFF7F5F810BDA06B4363FFF775FA0028DCD023685A69510605D51A69636A1A704E
:203F8000636A013363622268A06B136823F001031360202384F83D30C6E794F83D10602986
:203FA00015D1202184F83D1022645A69520605D51A69636A1A70636A013363622268204606
:203FC000136823F001031360FFF709FFAEE75A69500605D51A69636A1A70636A01336362B6
:203FE0002046FFF7DFF8A1E7E13D00080000FFFFF0B5044603688FB05A68C66A90F83E0091
:2040000094F83D101028C5B2C9B202D0402D40F0E5829F69586910F0010F07D1B6F52A0F32
:2040200002D0B6F12A4F51D10FB0F0BD96054DD5E26AB2F52A0F0CD10122E26294F83E20E9
:20404000402A11D1226D52B9626C02F0FE021A61EAE7E26AB2F12A4FF0D10822EDE7626C79
:2040600042F00102D2B2F2E72269B2F5804F1AD194F83D20212A626C11D102F0FE021A6171
:20408000626B0AB1926A2AB9A26B002ACCD0926A002AC9D05A6842F400625A60C4E742F036
:2040A0000102D2B2EBE7226D32B9626CD21102F0060242F0F002CAE7226D012AB4D1626CA0
:2040C000D21102F0060242F0F102C0E7060703D5960501D5626CE4E7860740F1F08096057F
:2040E00040F1ED8094F83E10E26A256B94F83D00C9B2222840F0DB80206D40B9402906D18D
:2041000000905A6900929B690093009B8CE7216D89B92069B0F5404F0DD101915A690192C2
:204120009A690192019A1A6842F480721A60236D0133236578E7618D89B251B902915A69F6
:2041400002929A690292029A1A6842F400721A6019E0618D89B2012949D112F5803F1BD1DC
:204160001A6822F480621A605A6812F400620CD01A6822F480621A60002203925A69039242
:204180009B690393039B0023D3E704925A6904929A690492049AD7E7082A1CD0202A1AD0D4
:2041A000122D0DD1012A16D11A6822F480621A60002205925A6905929B690593059BE2E7C4
:2041C000102AF1D8864941FA02F2D707ECD41A6842F48062EBE71A6822F480621A600022BE
:2041E00006925A6906929A690692069AACE7618D89B2022938D1102A03D87A49D140CE07E3
:2042000018D4196841F4006119600021079159690791996907910799196821F480611960E5
:2042200059680D05AFD5202A1BD8072A0ED8012AA9D111E0196841F4806119600021089173
:2042400059690891996908910899E9E7A2F10801654ACA40D00796D55A6842F480525A60DC
:2042600091E712F5803FE3E7196841F4806119605968090510D5202A16D8072A06D8012A00
:204280000AD15A6842F480525A6005E0A2F10801554ACA40D207F4D4002209925A690992D9
:2042A0009B690993099B6EE712F5803FE8E700220A925A690A929B690A930A9BB4E67F074D
:2042C00040F194805E6836053FF5AEAE070600F004063ED550053CD5002E3DD194F83D2063
:2042E000258D94F83E10D2B2E06AC9B2C5B9212A18D1082858D0202856D010F5803F53D08A
:204300005A6822F4E0625A6011232363002384F83E302023204684F83D30FFF704FD83E610
:20432000212A05D040297FF47FAE222A7FF47CAE628D92B21AB95A6822F48062ADE694F88C
:204340003E20402A16D120460FB0BDE8F040FFF7EDBC002E3FF468AE97057FF565AE212931
:2043600039D1E16A94F83D20212A7FF45DAE628D92B24AB1626A12F8011B19616262638DE8
:20438000013B9BB263854FE608290DD020290BD011F5803F08D0596821F4E06159601123A4
:2043A000236384F83E20B4E75A68204622F4E0625A601A6842F400721A6000232022236339
:2043C00084F83D2094F83E2084F83E30402AA4D1FFF7ABFC28E6402D7FF426AEB3E700BF99
:2043E000EBFFFEFF140001000101000159680E053FF51AAE450600F0040140F18680500522
:2044000040F18380002940F0838094F83D20222A7FF40AAEE06A628D92B2032A14D91A6992
:20442000636A1A70636A01336362638D013B9BB26385638D9BB2032B7FF4F6AD2268536838
:2044400023F480635360EFE5E56A022D3FF473AF012A3FF670AF0B9146F2A811794A1268BF
:20446000B2FBF1F202EB82020B920B9A013A0B920B99D1B9226C204642F0200222645A6863
:2044800022F4E0625A601A69636A1A70636A01336362638D013B9BB26385202384F83D30DD
:2044A00084F83E10FEF77EFEBEE51A6812F40072DBD1196821F480611960596821F4E06171
:2044C00059601969636A1970636A01336362638D013B9BB26385202384F83D3094F83E30FE
:2044E00084F83E20402B04D122632046FFF776FC9AE5082801D0202801D1002300E012237D
:2045000020462363FFF710FC8EE500293FF48CAD92057FF589ADE26A608D616A80B2042802
:2045200009D15A6822F480625A601B690B70636A0133636223E7608D80B203280CD1586877
:20454000042A20F480605860EFD0022AEDD01A6822F480621A60E8E7608D80B20228E4D118
:20456000042A33D007D8012A07D0022A2ED0186840F4007004E0102AF9D1186820F480607F
:2045800018601B690B70616A4B1C6362638D013B9BB2638523681B694B70636A21680133F8
:2045A0006362638D013B9BB263854B6823F440734B60202384F83D3094F83E30402B4FF0DD
:2045C000000384F83E3005D123638EE7186840F48060D5E7082A90D0202A8DE7206C20B31E
:2045E0000025586987072FD596052DD5226C02B19D6994F83D2002F02802282A18D15A685D
:204600002F0622F480625A604FF0000354BFE268A269C5F3800181F001012046C9B284F800
:204620003C3092B2FEF75FFDFEE49D695869D9E700220C9259690C919B6984F83C200C9376
:204640000C9BF1E428000020C60640F1B180950540F1AE8094F83D505A68EDB222F4E0629D
:204660005A6000220D925A690D921A6842F001021A600D9A1A6822F480621A605A681005BA
:2046800020D505F0F702222A4AD1A06B0268526892B26285628D92B21AB1226C42F00402B2
:2046A00022645A6822F400625A60FEF71BFF012808D0A06B794B4363FEF7CEFE10B1A06B6E
:2046C000436B9847638D9BB213B323685A69510709D51A69636A1A70636A01336362638D36
:2046E000013B9BB2638523685A69520609D51A69636A1A70636A01336362638D013B9BB2AC
:204700006385638D9BB21BB1236C43F004032364236C13B320460FB0BDE8F040FFF7C0BB98
:20472000606B0268526892B26285628D92B21AB1226C42F0040222645A6822F400625A6021
:20474000FEF7D0FE0128BDD0606B544B4363FEF783FE0028B6D0606BB2E72A2D06D1236394
:204760002823204684F83D30FEF706FD94F83D30282B0CD14A4B2022E36200232046236353
:2047800084F83D2084F83E30FEF7E1FC4CE4236B222B02D0222D7FF447AC00232022236307
:2047A00084F83D2084F83E302046FEF7E5FC3BE401F0F701212900F0040535D1070627D5A0
:2047C000560525D53DBB94F83D00628DC0B292B2002A3FF429AC626A12F8015B1D61626278
:2047E000628D013A92B26285628D92B2002A7FF41BAC29287FF418AC5A68204622F4806225
:204800005A602823216384F83D30FEF7C7FC0BE4002D3FF409AC95057FF506AC628D92B277
:20482000002A3FF401ACA5E5400627D5510525D53DBB94F83D20618DD2B289B200293FF468
:20484000F3AB1969636A1970636A01336362638D013B9BB26385638D9BB2002B7FF4E4AB51
:204860002A2A7FF4E1AB2268536823F48063536022232363282384F83D3095E7002D3FF418
:20488000D3AB92057FF5D0AB628D92B2002A3FF4CBAB1A69636A1A7049E600BFE13D000820
:2048A0000000FFFFF8B5036804465F695E6890F83E2017F48075D2B20AD016F4807507D0F0
:2048C0006FF4807101255961196841F400411960B80506D5F10542BF6FF4007145F0020595
:2048E0005961780536D5F10534D5608D94F83D10202AD4F830C080B2C9B25FD100285DD178
:2049000001F0F700212804D0282957D1BCF1210F54D194F83D20E16AD2B2082901D0202914
:204920002AD1282A28D12E4A2046E2625A6822F4E0625A606FF480625A611A6822F48062C1
:204940001A6000232022236384F83D2084F83E30FEF7FDFB3A053FD5F3053DD56FF4006220
:20496000236845F008055A61236C20461D432564BDE8F840FFF794BA212A1BD11849E162D5
:2049800022630021202284F83D2084F83E105A6822F4E0625A606FF480625A611A6822F420
:2049A00080621A605A69100648BF19612046FEF7F5FBCFE76FF480625A61CBE76FF480614A
:2049C000102A596145F0040501D0402AC2D11A6842F400721A60BDE7002DC5D1F8BD00BF58
:2049E0000000FFFF90F83D007047006C704700002DE9F341054638B30368DB0710D42B68D6
:204A00009F075ED42B68190700F195802B685A0700F1C180EB69002B40F02C81002029E05A
:204A2000904C636803F00C03042B07D0636803F00C03082B0AD16368DE0307D523689C033A
:204A4000DDD56B68002BDAD1012013E06B68B3F5803F12D1236843F480332360FEF73CFCA5
:204A6000064623689803CAD4FEF736FC801B6428F7D9032002B0BDE8F0819BB9236823F427
:204A800080332360236823F480232360FEF724FC064623689903B2D5FEF71EFC801B6428D3
:204AA000F7D9E6E7B3F5A02F236803D143F480232360CFE723F480332360236823F48023DE
:204AC000CBE7684C636813F00C0F07D0636803F00C03082B10D16368DA030DD423689B0719
:204AE00002D52B69012BAFD123686A6923F0F80343EAC203236085E72A695B4B6AB10122DB
:204B00001A60FEF7E9FB064623689F07ECD4FEF7E3FB801B0228F7D9ABE71A60FEF7DCFBC5
:204B20000646236898077FF56DAFFEF7D5FB801B0228F6D99DE7AA694A4E4B4BE2B101229B
:204B4000C3F88024FEF7C8FB0446736A9B070DD54FF4FA52454B1B68B3FBF2F3019300BF0B
:204B6000019B5A1E0192002BF9D14FE7FEF7B4FB001B0228E9D97CE7C3F88024FEF7ACFB5A
:204B80000446736A9F077FF541AFFEF7A5FB001B0228F6D96DE7334CE369D80024D4012724
:204BA000E36943F08053E361E36903F080530093009B2F4E3368D90518D5EB68012B26D1C6
:204BC000236A43F001032362FEF786FB41F288380646236A9B073FD5002F3FF41BAFE3691C
:204BE00023F08053E36115E70027E2E7336843F480733360FEF770FB80463368DA05DCD4F7
:204C0000FEF76AFBA0EB08006428F6D931E7ABB9236A41F2883823F001032362236A23F014
:204C200004032362FEF758FB0646236A9807D3D5FEF752FB801B4045F7D91AE7052B236A90
:204C400003D143F004032362BAE723F001032362236A23F00403B6E7FEF73EFB801B4045F2
:204C6000B7D906E7001002400000424228000020007000402A4C626802F00C02082A3ED069
:204C80000022022B274B1A662CD1FEF725FB06462368990120D42B6AB3F5803F05D16268C0
:204CA000A96822F400320A436260696A62680B4322F474121343012263601A4B1A66FEF7EF
:204CC0000BFB054623689A013FF5A8AEFEF704FB401B0228F6D9CCE6FEF7FEFA801B022827
:204CE000D6D9C6E6FEF7F8FA054623689B017FF595AEFEF7F1FA401B0228F6D9B9E6012B4A
:204D00003FF4A2AE60682B6A00F480329A427FF49BAE6B6A00F47010C01A18BF0120A9E6CB
:204D200000100240000042420D4A536803F00C01082912D10B48C3F38341DB03405C09D552
:204D40005368094AC3F340435043084AD35CB0FBF3F07047064B584370470348704700BF4F
:204D600000100240D697000800127A00D497000800093D002DE9F0410D46044610B9012059
:204D8000BDE8F081444A136803F007038B4228D321688E0730D4CA0743D43F4A136803F02E
:204DA0000703AB4265D822683C4D12F0040F6CD1130706D56B68226923F4605343EAC2034B
:204DC0006B60FFF7B1FF6B68354AC3F30313D35CD840344B1860344B1868FEF73BFA0020BD
:204DE000CEE7136823F007030B431360136803F007038B42C3D1CBE7284B11F0040F1EBFB6
:204E00005A6842F4E0625A60080742BF5A6842F460525A605A68A06822F0F00202435A605D
:204E2000B9E762681D4E012A33681AD113F4003FA5D0736841F2883823F003031343736021
:204E4000FEF74AFA07467368626803F00C03B3EB820FA2D0FEF740FAC01B4045F3D9032006
:204E60008EE7022A02D113F0007FE1E713F0020FDEE7136823F007032B431360136803F0B4
:204E80000703AB427FF47BAF8DE76B68E16823F4E0630B436B608BE7002002400010024055
:204EA0003C9800082800002008000020044B054A5B68C3F30223D35C034A1068D8407047A7
:204EC000001002403498000828000020044B054A5B68C3F3C223D35C034A1068D8407047A5
:204EE0000010024034980008280000200F2303600B4B5A6802F0030242605A6802F0F00258
:204F000082605A6802F4E062C2605B68DB0803F4E0630361034B1B6803F007030B6070475F
:204F20000010024000200240036A026A70B522F001020262446882690D6822F073022A4346
:204F40008D6823F002032B430A4DA8420BD1CD6823F008032B4324F44074D1E9055635439F
:204F600023F004032C43446082614A684263036270BD00BF002C0140036A026A70B522F4F8
:204F8000807202624468C2690D6822F073022A438D6823F4007343EA05230B4DA8420DD187
:204FA000CD6823F4006343EA052324F44054D1E90556354323F4806344EA05144460C261AC
:204FC0004A68C263036270BD002C0140036A026A30B522F4805202624468C2690D6822F48F
:204FE000E64242EA05228D6823F4005343EA0533064DA84202BF4D6924F4804444EA85141B
:205000004460C2614A680264036230BD002C014090F83D30012B1CD102230F4A80F83D3081
:20502000036893420AD0B3F1804F07D0A2F59432934203D002F58062934204D19A6802F090
:205040000702062A03D01A6842F001021A60002070470120704700BF002C014090F83C2054
:205060000346012A4FF0020009D01A6883F83D0051610020012283F83C0083F83D2070472D
:2050800070477047036870B5DD681E690446B1070DD5AA070BD56FF002021A610122027757
:2050A0009B699B0769D001F02CFA00232377710710D56A070ED56FF00402236820461A61BB
:2050C000022222779B6913F4407F5CD001F019FA0023237733070FD528070DD56FF00802C4
:2050E000236820461A6104222277DB69990750D001F007FA00232377F20610D5EB060ED521
:205100006FF01002236820461A6108222277DB6913F4407F43D001F0F4F900232377F00740
:2051200008D5E90706D56FF00102236820461A6101F0C4F9320608D52B0606D56FF0800249
:20514000236820461A6100F004FB700608D5690606D56FF04002236820461A61FFF791FFC4
:20516000B20622D5AB0620D56FF0200223682046BDE870401A6100F0EBBA01F0C0F92046F3
:20518000FFF77EFF91E701F0BAF92046FFF778FF9EE701F0B4F92046FFF772FFAAE701F03B
:2051A000AEF92046FFF76CFFB7E770BD174A036890420AD0B0F1804F07D0A2F594329042C8
:2051C00003D002F58062904207D14A6823F070031343CA6823F4407313434A6923F0800350
:2051E000134303608B68C3620B688362074B984204BF0B690363012343610369DB0742BFA6
:20520000036923F001030361704700BF002C014010B5044630B390F83D3003F0FF021BB915
:2052200080F83C2001F006FF0223206884F83D30211DFFF7BBFF0123002084F8463084F86E
:205240003E3084F83F3084F8403084F8413084F8423084F8433084F8443084F8453084F8E2
:205260003D3010BD0120FCE7036A026A70B522F010020262446882690D6822F4E64242EAF4
:2052800005228D6823F0200343EA05130B4DA8420DD1CD6823F0800343EA051324F440648B
:2052A000D1E90556354323F0400344EA8504446082614A688263036270BD00BF002C014078
:2052C00010B590F83C300446012B1DD0082A17D007D862B1042A0FD00120002384F83C306E
:2052E00010BD0C2AF8D10068FFF770FE02E00068FFF71AFE0020F0E70068FFF7B5FFF9E7D5
:205300000068FFF739FEF5E70220E9E738B590F83C300446012B4FD00120082A84F83C00A9
:205320003AD006D8BAB1042A26D0002384F83C3038BD0C2AF9D12068FFF748FEC3690A6993
:2053400043F40063C361C36923F48063C361C36943EA02232EE02068FFF7E6FD83690A69F9
:2053600043F008038361836923F0040383618369134383610020D8E72068FFF775FF83693E
:205380000A6943F400638361836923F480638361836943EA0223ECE72068FFF7EDFDC369AD
:2053A0000A6943F00803C361C36923F00403C361C3691343C361DDE70220B9E770B5056AEE
:2053C000046A114E24F001040462B042846916D0B0F1804F13D0A6F59436B0420FD006F538
:2053E0008066B0420BD044F0010263F3071201F00A0125F00A0319438261016270BD24F053
:2054000003042243F1E700BF002C0140F8B590F83C300546012B0C4600F081800120082A6E
:2054200085F83C005BD006D842B3042A35D0002385F83C30F8BD0C2AF9D1D1E900272B684D
:20544000CE68186A196A120321F480511962D96920F4005021F4407141EA072102F4005294
:2054600066F30F310243D9611A62DA69A16822F44062DA61DA6942EA01224EE02868CB68D6
:2054800006C9FFF79BFF8369A26823F00C0383618369134383610020C9E72B68D1E9002747
:2054A000186ACE68196A120121F010011962996920F0A00021F4407141EA072102F0A002A2
:2054C00066F30F31024399611A629A69A16822F440629A619A6942EA01229A61DBE72B6817
:2054E000D1E90021186A1E6AE76826F480761E62DE69120226F00306314320F4007002F480
:20550000007267F307110243D9611A62DA69A16822F00C02DA61DA690A43DA61BBE7022076
:2055200088E710B50124036A01F01F018C4023EA04030362036A8A401A43026210BD00008A
:2055400008B529B990F83E30012B1DD001202EE0042907D190F83F30012BF7D1022380F8E1
:205560003F3014E0082907D190F84030012BEDD1022380F840300AE090F84130012BE5D10B
:20558000022380F8413002E0022380F83E3000680122FFF7C6FF0F4B984209D0B0F1804F4D
:2055A0000BD1836803F00703062B0DD1002008BD436C43F400434364F3E7074B9842F0D09D
:2055C00003F580639842ECD0036843F001030360ECE700BF002C014000040040FFF7B0BFAD
:2055E00008B5034641BB90F83E0093F84220C0B20128D2B24DD1012A1DD1022291BB83F8B5
:205600003E2083F8422018680122FFF78AFF224B98420AD0B0F1804F07D0A3F5943398428C
:2056200003D003F5806398422ED1836803F00703062B29D1002008BD042905D190F83F0021
:2056400093F84320C0B2D3E708290BBF90F8400093F8410093F8442093F845200CBFC0B285
:20566000C0B2C5E7042904D183F83F2083F84320C9E708290BBF83F8402083F8412083F875
:20568000442083F84520BEE7036843F001030360D0E70120CFE700BF002C014010B5042475
:2056A000036A01F00F018C4023EA04030362036A8A401A43026210BD08B529B990F84230D9
:2056C000012B1DD001203EE0042907D190F84330012BF7D1022380F8433014E0082907D171
:2056E00090F84430012BEDD1022380F844300AE090F84530012BE5D1022380F8453002E0F6
:20570000022380F8423000680422FFF7C7FF436C43F4004343640C4B98420AD0B0F1804FE5
:2057200007D0A3F59433984203D003F58063984204D1836803F00703062B03D0036843F072
:2057400001030360002008BD002C0140FFF7B4BF70477047026802F10C0353E8003F23F4BC
:2057600090730C3242E8003102680029F2D102F1140353E8003F23F0010302F1140C4CE855
:2057800000310029F3D1036B012B0BD102F10C0353E8003F23F0100302F10C0C4CE8003163
:2057A0000029F3D1202380F8423000230363704710B504460368C1681A6922F440520A4374
:2057C0001A6182680069D9680243606921F4B05121F00C0102430A43DA605A69A16922F4C9
:2057E00040720A435A610E4A934215D1FFF76EFB19234343626820689200B3FBF2F36422BE
:20580000B3FBF2F102FB11331B013233B3FBF2F303EB0113836010BDFFF748FBE8E700BF29
:2058200000380140F7B505460C4617461E462A68136834EA030301D1002021E0701CF7D06E
:20584000FDF74AFDC01B86421CD3DEB12B68DA685107ECD5802CEAD0402CE8D01A681207D9
:20586000E5D5002401941A68284601925B680193019BFFF76FFF082301206B6485F84040C3
:2058800003B0F0BD0320FBE7704710B5044648B390F8413003F0FF021BB980F84020FFF753
:2058A000F3FF2423226884F84130D368204623F40053D360FFF77CFF236800201A6922F445
:2058C00090421A615A6922F02A025A61DA6842F40052DA602023606484F8413084F84230D9
:2058E000606310BD0120FCE710B5044668B390F8413003F0FF021BB980F84020FFF7C4FF98
:205900002423226884F84130D368204623F40053D360FFF74DFF236800201A6922F4904233
:205920001A615A6922F022025A615A6942F008025A61DA6842F40052DA602023606484F8F7
:20594000413084F84230606310BD0120FCE72DE9F843984690F841300446202B0E461746E6
:205960003FD100293FD0002A3DD021230025456480F84130FDF7B0FCA3688146B3F5805FB4
:20598000A784E78403D123690BB935461E46E38C9BB253B943464A4640212046FFF742FF8F
:2059A000202350B984F841300AE043464A4680212046FFF737FF28B12023032084F841304C
:2059C000BDE8F88322684EB935F8023BC3F308035360E18C013989B2E184D8E716F8013BE8
:2059E000F6E70220ECE70120EAE790F84130202B10D189B182B1C28482840023212201623C
:205A00000168436480F84120CA68184642F08002CA607047022070470120704708B50023E7
:205A2000406AC385C38401F067FD08BD704790F8423007B5222B42D181680268B1F5805F6E
:205A4000836A3FD1016900293FD15268C2F3080223F8022B8362C38D013B9BB2C385002BB4
:205A60002DD10268D16821F02001D160D16821F48071D160516921F001015161202280F879
:205A800042204363026B012A026828D1036302F10C0353E8003F23F0100302F10C0C4CE8BC
:205AA00000310029F3D11368DB0605D501911368019353680193019B818DFFF7B7FF03B099
:205AC0005DF804FB39B9016929B95268D2B21A70836A0133BEE7526802F07F02F7E701F0AA
:205AE00005FDECE7036873B51A6804461607D9685D6908D1960668D58D0666D502B0BDE877
:205B00007040FFF794BF05F0010001F4907505435BD0D60705D5CD0542BF636C43F0010399
:205B20006364530704D518B1636C43F002036364960704D518B1636C43F0040363641507A9
:205B400007D501F0200303431EBF636C43F008036364636C002B32D0920604D58B0602D589
:205B60002046FFF764FF266820467369626C03F0400302F0080253EA020522D0FFF7EAFD83
:205B800073695E0618D5226802F1140353E8003F23F04003143242E800310029F3D1E06B9B
:205BA00050B1744B4363FDF757FC40B1E06B436B02B0BDE870401847204601F09DFC02B046
:205BC00070BD01F099FC6564F9E7206B012840F09480D50640F19180C80640F18E80002225
:205BE00001921A6801925A680192019A5A6952064DD5E16B0A68526892B2002ADFD0A08D0E
:205C00009042DCD9E2858A69202A36D003F10C0252E8002F22F4807203F10C0040E8002197
:205C20000029F3D103F1140252E8002F22F0010203F1140040E800210029F3D103F11402A7
:205C400052E8002F22F0400203F1140040E800210029F3D1202284F84220216303F10C02A3
:205C600052E8002F22F0100203F10C0040E800210029F3D1E06BFDF7CFFB02236363E38DFD
:205C8000A18DC91A89B22046FFF7D0FE97E7E28DE18D92B289B2002991D0A18D891A89B21E
:205CA00000298CD003F10C0252E8002F22F4907203F10C0545E800200028F3D103F1140294
:205CC00052E8002F22F0010203F1140545E800200028F3D1202284F84220206303F10C025B
:205CE00052E8002F22F0100203F10C0545E800200028F3D102236363C5E7160628D50D0616
:205D000026D594F84120212A7FF459AFA168226AB1F5805F17D12169A9B932F8021BC1F3EC
:205D2000080159602262E28C013A92B2E284002A7FF445AFDA6822F08002DA60DA6842F0B5
:205D40004002DA603BE7511C216212785A60EAE750067FF534AF4A067FF531AFDA682046A7
:205D600022F04002DA60202384F8413001F0C1FB25E700BF1D5A000890F84030012B11D069
:205D80002423026880F84130D36823F00C0343F00803D360202380F84130002380F8403064
:205DA000184670470220704790F84030012B11D02423026880F84130D36823F00C0343F0C6
:205DC0000403D360202380F84130002380F84030184670470220704790F8412090F84200B1
:205DE000104370470023C285436422238285026980F84230816203681AB1DA6842F4807264
:205E0000DA605A69002042F001025A61DA6842F02002DA60704770B590F84260202E07D179
:205E200041B13AB100240463FFF7DCFF204670BD0220FCE70120FAE7836810B504462BB1B9
:205E40000322014698470023C4E9023310BD4B1E032B00D9FEE78900081F70470139435C90
:205E600013F0100004D0022916D80C4A32F81100DB0712D503290FD8DFE801F00205080BE3
:205E800040F00100704740F01000704740F48070704740F480507047FEE77047EE97000864
:205EA0000139032900D9FEE7014B585C704700BFEA9700080139032900D9FEE7014B585C9B
:205EC000704700BFE69700082DE9F0410E460446FFF7BDFF06F1060805463146204604EB14
:205EE0000818FFF7DDFFD8F808302BB1C24323691A61DA680243DA60771E04EB47039B880E
:205F00000B2B49D8DFE803F051181818060618184A4A4A2AE35DDE0604D5294604F1100022
:205F2000FFF714FCE35DD80736D5294604F11000BDE8F041FFF752BBE35DD90604D529467D
:205F400004F11000FFF7B8FBE35DDA0724D5294604F11000BDE8F041FFF7F2BA294604F129
:205F60001000FFF73DFB31462046FFF7A3FF014606462046FFF772FF25692B6A1843D8F8C0
:205F80000830286243B131462046FFF789FFC3432B61EB681843E860BDE8F081294604F1EE
:205FA0001000BDE8F041FFF71BBB23691B68DB07F2D404F11000BDE8F041FFF729B870B5A1
:205FC000012504462946861C36F8023F23B129462046FFF779FF00210135052DF4D1A36E5B
:205FE0003BB16FF0010223691A61DA6842F00102DA6049B123691B68DB0705D404F11000D2
:20600000BDE87040FFF704B870BD00002DE9F0438DB0044698460F46FFF719FF4FF6FF7384
:206020001646059305462369C0B95B6B002206930123CDE902329DF85030CDE909220792FE
:2060400008920B92019204930B2E1DD8DFE806F00F1545484A5355575B596264042801D182
:206060009B6BE3E708280CBFDB6B1B6CDEE705922A4605A904F1100004E010232A460593EA
:2060800005A9E018FFF71CF9013F04EB47039E8006B3B8F1FF3F1DD0404601F00DF8A842C5
:2060A00064D140463249083E00F0A0FE032E05D8404601F017FF002101F0DAFF40462C4955
:2060C00000F0CEFE10F4801F0CBF01221022E35D1343E3550DB0BDE8F08320230593C7E715
:2060E0003023FBE760232A4605A904F110000593FFF70CF9C8E77023F5E75023EEE7402369
:20610000ECE7022301932A4601A904F11000FFF77DF9B9E70A23F5E74046154900F0A0FE4D
:2061200010F4801000D0FEE7012304F110092A46019001A948460293FFF768F939462046DA
:20614000FFF7B8FE431EE25C014642F00102E2540B2204EB43039A8002232046CDE9013351
:20616000FFF775FE01A902464846D0E7FEE700BF54990008013903299ABF00EB41008088F3
:206180000020704701211030FEF768BF0369186800F00100704710B502460C46FFF7F6FFCC
:2061A00080B9CB68DB070ED5CB68104623F00103CB60FFF7E7FF6FF001032361E36843F0A2
:2061C0000103E36010BD1046BDE81040FFF7DABF0B4B98420BD0B0F1804F0AD0A3F594331D
:2061E000984208D003F58063984206D0FEE70020704701207047022070470320704700BF5C
:20620000002C0140024670B5044652F8100FFFF7DFFF0546104600F09FFE0023084A04F185
:20622000600642F82530E36004F1B005B54204D0103D2846FAF72FF8F8E7204670BD00BFAD
:2062400098050020F8B504460846FFF7C1FF236903B1FEE71B4D04F10C0245F820200E2249
:2062600004F110063046C4E90C33C4E90E33C4E91033C4E91623216184F82C30A36484F810
:206280004C3084F84D30E46000F022FE04F1600504F1B00728461035FFF7CEFDBD42F9D1F2
:2062A00000234FF6FF72C4E90033C4E90632C4E90833A360636180233046A362BDE8F84096
:2062C000FEF7A6BF9805002010B586B014220446002101A802F034F90023694601A8009335
:2062E000FEF704FE206900F0CDFE012802D002280FD0FEE7049CFEF7D9FDB4F5C06F05D062
:206300000BD824F48074B4F5806F00D1400006B010BD059CFEF7DAFDEFE7B4F5E06FF4E74C
:20632000012A38B505460C460BD0022A16D004B1013C29692846CC62EC61BDE83840FFF73B
:206340002ABFFFF7C1FF084BB0FBF3F044432A69230C93620133B4FBF3F4E8E7FFF7B4FF3D
:20636000B0FBF4F4F3E700BF40420F00F8B5054614461A46FFF76BFD2B69822A9E6A0746BB
:2063800006F1010629D01FD8102A11D852BB4FF6FF722969CB6A934203D1B4F5803F08BF8A
:2063A0001C4637BB4C632846BDE8F840FFF7F3BE812AECD12846FFF787FF124BB0FBF3F0AB
:2063C0006043B0FBF6F4E2E7832AE0D1DB6A03FB04436424B3FBF4F4D9E72846FFF774FF1F
:2063E0006643EEE7DB6A03FB044301249440013CF0E7042F01D18C63D5E7082F0CBFCC63A7
:206400000C64D0E740420F00034B186810B10430FEF738BE704700BF98050020FFF7F4BF3A
:20642000034B586810B10430FEF72CBE704700BF98050020034B986810B10430FEF722BE2F
:20644000704700BF98050020034BD86810B10430FEF718BE704700BF980500200022C0E9BD
:206460000022C0E902227047F8B504460E4600F1600500F1B00728461035FFF7EFFFBD4297
:20648000F9D10023204631462361FFF7DBFE2046F8BD826810B50AB902F048FCC368BDE84C
:2064A0001040184708B500B9FEE700F00FFD0068836E13B16030FFF7ECFF08BDFFF7F2BFDC
:2064C00010B500B9FEE7037F013B072B10D8DFE803F004140F100F0F0F12012400F0F6FC4A
:2064E0000068063400EB041083680BB1FFF7D1FF10BD0324F2E70424F0E70224EEE7FFF7D1
:20650000DFBFFFF7DDBF01F0ABBE01F0B1BE000086B0042841D8DFE800F003101C283400D4
:206520001F4B20489A6942F004029A619B6903F004030193019B06B07047194B1A489A69EF
:2065400042F008029A619B6903F008030293029BF1E7134B15489A6942F010029A619B69F7
:2065600003F010030393039BE5E70D4B10489A6942F020029A619B6903F020030493049BC3
:20658000D9E7074B0B489A6942F040029A619B6903F040030593059BCDE70020CBE700BF6D
:2065A0000010024000080140000C01400010014000140140001801402DE9F3478A46244967
:2065C00099469046064600F029FCFFF701FE214F054657F8203073B9B020FFF794FF1C496C
:2065E0000446304600F01AFC01462046FFF73CFF57F825301C60164930461C6800F030FC62
:20660000C0F3C43529462046FFF7B4FD0428074607D0002304220093294633462046FFF7E2
:20662000F5FC022251462046FFF77AFE4B46424629462046FFF79AFE042F05D0204602B03E
:20664000BDE8F047FFF7BBBC02B0BDE8F08700BF5499000898050020F8B51349064600F06D
:20666000DDFBFFF7B5FD114F054657F8203073B9B020FFF748FF0C490446304600F0CEFB49
:2066800001462046FFF7F0FE57F825301C601C6844B12046FFF7B6FD2046BDE8F840B021AD
:2066A000FFF733BFF8BD00BF5499000898050020FCF712BE704708B5FCF702FEFCF797FE1A
:2066C000FFF7F8FF08BD70470F4B84B0DA6942F08052DA61DA6902F080520192019A9A6909
:2066E00042F001029A619A6902F001020292029A5A6942F040025A615B6903F040030393C0
:20670000039B04B0704700BF001002400C4BD3F8FC20D2015EBFD3F8FC2042F08072C3F86B
:20672000FC200022074B5A601A6842F001021A6000BF00BF00BF5868B0FA80F040097047C7
:2067400000ED00E0001000E008B5FFF7BDFFFFF7DDFFFCF7A3FDFFF7B6FF00F05DFFBDE80C
:2067600008400148FCF748BE200000200023C0E90033C0E9023370472DE9F04316460027EF
:206780000A468BB0012A07F101046ED1CDE902130023FF2998BF02461D461C464FF0010C41
:2067A00088BF021D0CFA03FE714505D11D46FF294FEA830488BF203C0133102BF2D10F238E
:2067C0001268A34013400822A240934250D10123C268AB4093430CBF012302230493032327
:2067E000142402A90593FCF781FE0023FFB27C43DFF88480D6F80890043406AD06934444CC
:20680000C5E901330993B9F1000F33D0022231462846C847D6E9029C95E8030014267E434E
:20682000CDE9000108EB0603043393E8030085E80300DDE9000183E80300A3682846089337
:20684000E368C4F80890C4F80CC00993F9F723FD0022062118F90600FCF756FD18F90600A8
:20686000FCF782FD0BB0BDE8F0832746520889E70023B3E7CC46CFE7A805002000230128FE
:2068800003F101020AD11422DBB25343054A181D1044816829B11A44136918471346400858
:2068A000EDE77047A80500200120FCF7F3BE0220FCF7F0BE0420FCF7EDBE0820FCF7EABE73
:2068C0001020FCF7E7BE08B52020FCF7E3FE4020FCF7E0FE8020FCF7DDFE4FF48070FCF75A
:2068E000D9FEBDE808404FF40070FCF7D3BE38B506244FF48065A8B2FCF7CCFE013C4FEAD1
:206900004505F8D138BD0000344A08B51046062300F8043BFFF72AFF072302F118001375A2
:20692000FFF724FF082302F12C0082F82830FFF71DFF092302F1400082F83C30FFF716FFC0
:206940000A23172102F1540082F85030FFF70EFF02F1680082F86410FFF708FF02F17C00D9
:2069600082F87810FFF702FF02F1900082F88C10FFF7FCFE02F1A40082F8A010FFF7F6FEEA
:2069800082F8B410282102F1B800FFF7EFFE02F1CC0082F8C810FFF7E9FE02F1E00082F8A7
:2069A000DC10FFF7E3FE02F1F40082F8F010FFF7DDFE02F5847082F80411FFF7D7FE02F5A6
:2069C0008E7082F81811FFF7D1FEBDE8084002F5987082F82C11FFF7C9BE00BFA8050020A5
:2069E00038B5054CA4F5A075143C201DF9F753FCAC42F9D138BD00BFE80600207B4B82B06D
:206A00009A69013842F001029A619B6903F001030193019B23282CD8DFE810F024002D0078
:206A200034003B00400047004C00530058005F0068006D0074007D008200890092009B000C
:206A4000A000A700B000B500BC002B002B002B00C100C8002B002B002B002B00CD00D20079
:206A6000D900E000624A536843F0E06343F00103536002B070475E4A536823F0010343F080
:206A8000E063F5E75A4A536843F0E06343F00203EEE7574A536823F00203F0E7544A536851
:206AA00043F0E06343F00403E2E7514A536823F00403E4E74E4A536843F0E06343F008031B
:206AC000D6E74B4A536823F00803D8E7484A536843F0E06343F03003CAE7454A536823F095
:206AE000300343F0E06343F01003C1E7404A536823F03003C3E73E4A536843F0E06343F0DE
:206B0000C003B5E73A4A536823F0C00343F0E06343F04003ACE7364A536823F0C003AEE7DC
:206B2000334A536843F0E06343F44073A0E7304A536823F4407343F0E06343F4007397E799
:206B40002B4A536823F4407343F0E06343F480738EE7274A536823F4407390E7244A536890
:206B600043F0E06343F4406382E7214A536823F4406343F0E06343F4006379E71C4A5368EB
:206B800023F440637BE71A4A536843F0E06343F480536DE7164A536823F480536FE7144A2D
:206BA000536843F0E06343F4004361E7104A536823F4004363E70E4A536823F0E06357E782
:206BC0000B4A536823F0E06343F0807350E7084A536823F0E06343F0007349E7044A5368B0
:206BE00023F0E06343F0806342E700BF001002400000014091FAA1F3B3FA83F370B50D0E2C
:206C00000F2691FAA1F1B1FA81F144599B0006FA03F3890024EA03048A402243425170BD4A
:206C200091FAA1F3B3FA83F370B50D0E042691FAA1F1B1FA81F144599B0006FA03F38900B7
:206C400024EA03048A402243425170BD431C04D00C3151F80C3C5A1C01D10020704783424B
:206C600001F10C01F5D1012070470000431C2DE9F34106460F4600D1FEE7594B00F00F02D2
:206C8000C0F3031001F0070853F82240FFF740FCB8F1010F054615D194FAA4F3B3FA83F31D
:206CA0000321200E2A589B0001FA03F322EA030294FAA4F3B3FA83F39B00994011432950DA
:206CC000012213E0C7F30620B8F1030F0AD801A353F828F0E76C0008C16C00084B6D0008CA
:206CE000596D0008FEE7FFF789FE08222146284608F1FF38FFF77EFFB8F1010F06D817F024
:206D0000080218BF04222146FFF78AFF94FAA4F2230EB2FA82F2E9580F239200934094FAAB
:206D2000A4F2B2FA82F2C7F301170B409200012F23FA02F312D0022F3BD0082B21D1042243
:206D400021462846FFF756FF1BE07F2801D10922CCE7FFF753FEFAE70022C7E7042B04D1C5
:206D6000082221462846FFF745FF230A93FAA3F3B3FA83F20123E968934021EA14210B4392
:206D8000EB60184B9A6942F001029A619B6903F001030193019BA6F10D03012B14D8124ACC
:206DA000536823F0E06343F08063536002B0BDE8F081042B04D1082221462846FFF71AFF1F
:206DC000EB6823EA1423DBE70F2E02D0133E012EECD8054A536823F0E06343F00073E4E736
:206DE000F49700080010024000000140431C06D17047834202D18968FFF738BF0C310B685A
:206E00005A1CF6D1FEE70B685A1C01D100207047834201D1486870470C31F4E7431C01D078
:206E2000FFF7F1BF002070474B6813B94FF0FF307047834201D1086870470C31F4E708B1A2
:206E4000FFF7F2BF4FF0FF30704703460868421C00D17047984201D1886870470C31F5E75B
:206E6000431C01D0FFF7F1BF704703468B42084604D01BB100290CBF184600207047000058
:206E80000F4B1A6842F001021A6059680D4A0A405A601A6822F0847222F480321A601A68FD
:206EA00022F480221A605A6822F4FE025A604FF41F029A604FF00062034B9A60704700BF51
:206EC000001002400000FFF800ED00E00438704703681D4A84B093420BD11C4B9A6942F452
:206EE00000629A619B6903F400630093009B04B07047B3F1804F0BD103F50433DA6942F04B
:206F00000102DA61DB6903F001030193019BEEE70F4A93420AD10D4BDA6942F00202DA61DE
:206F2000DB6903F002030293029BE0E7094A9342DDD1064BDA6942F00402DA61DB6903F008
:206F400004030393039BD2E7002C01400010024000040040000800400368124A934206D17F
:206F600002F56442936923F4006393617047B3F1804F05D10C4AD36923F00103D361704776
:206F80000A4A934205D102F50332D36923F00203F4E7074A9342F2D102F50232D36923F034
:206FA0000403EBE7002C0140001002400004004000080040431C10D00C4B984210D007D87E
:206FC000B0F1804F0ED0A3F5806398420CD0FEE7074B9842FBD1192070476FF00D00704742
:206FE0001E2070471C2070471D20704700080040002C0140431C10D00C4B984210D007D8D1
:20700000B0F1804F0ED0A3F5806398420CD0FEE7074B9842FBD11B2070476FF00D007047FF
:207020001E2070471C2070471D20704700080040002C014038B50446FFF74AFF0068FFF7EB
:20704000B9FFD4E91212FCF75FF92068FFF7B2FFFCF78AF922681046FFF7CCFF0546104665
:20706000FFF7A8FF85420BD0D4E912122846FCF74BF92068FFF7BEFFBDE83840FCF774B9D3
:2070800038BD0000431C0CD0094B98420BD007D820F48063B3F1804F07D0064B984204D098
:2070A000FEE700207047022070470120704700BF002C01400008004008B50649FFF7D0FE1F
:2070C000C0F3C430431E032B00D9FEE78000043808BD00BF549900082DE9F04F87B098461D
:2070E000109B04468A46406D664991460193FFF795FE65498346A06DFFF790FE634906467B
:20710000E06DFFF78BFE62490546206EFFF786FE0746BBF1000F00F0B180A26D013202D068
:20712000002E00F0AB80E26D013202D0002D00F0A580226E013202D0002F00F09F80314626
:207140005846FFF792FE0346206020B90146FFF78CFE0346206029461846FFF786FE394613
:207160002060FFF782FE2060002800F08780494B98424CD103F55843DA6842F48042DA60E8
:20718000DA6822F48042DA609A6942F480429A619B6903F480430393039B2523A4F864303B
:2071A0003849606DFFF722FE1EB13749A06DFFF71DFE2DB13549E06DFFF718FE4FF4807511
:2071C0002FB13349206E45F40075FFF70FFE94F86520314B271D43F8227023680022C4E91C
:2071E000013A019B94F96400C4E904380C230121C4E90635C4F80C902262FCF785F83846DB
:20720000002E36D107B0BDE8F04FFEF76DBB234B984215D103F5E6331A6942F400321A61DC
:207220001A6922F400321A61DA6942F40032DA61DB6903F400330493049B4FF49373ADE7A1
:20724000174B9842ACD103F5E4331A6942F480221A611A6922F480221A61DA6942F48022BF
:20726000DA61DB6903F480230593059B40F2272394E707B0BDE8F04FFEF707BB07B0BDE818
:20728000F08F00BF0C990008C4980008889800084C98000800380140E80600200044004080
:2072A0000048004010B4019C18B1019410BCFFF713BF10BC704700000A4A0B4B926813B504
:2072C00053F8224009492046FFF7A8FD40B1002307481A4644654FF416510093FFF7FCFE15
:2072E00002B010BDE89B0008289C00080C9900082C00002008B5074B90F8652053F8220036
:20730000FEF76AFD00F02200A0F122035842584108BD00BFE806002008B5074B90F8652068
:2073200053F82200FEF758FD00F02100A0F121035842584108BD00BFE80600202DE9F843BA
:2073400006460C46FBF7C8FF274D074695F86530022B2ED9254A264B9268264953F8228089
:207360004046FFF75BFDF0B900242046BDE8F88359F8232052B140461E49FFF74FFD95F893
:20738000653059F823201268824210D00133DBB2022B85F86530EBD9FFF78EFF95F865303D
:2073A000022B06D9E0E70023DFF84C90F0E7022BF2D8114A52F82350A5F104084046FFF720
:2073C000ABFF48B94FF47A7331462846A2B2FEF7BEFA0028C8D1C8E7FBF77EFFC01BB0F58D
:2073E0007A7FEBD3C0E700BF2C000020E89B0008289C00080C990008E806002070B50E4699
:20740000054610B94FF0FF3070BDFFF773FF04460028F7D1294611F8663F0122337095F8AB
:207420006500034B53F82000FEF7F5FC2046EBE7E806002038B50D460446B8B1FFF75AFFC0
:20744000A0B994F96400E564FBF79CFF94F86500074B04F1660153F820000122FEF7DBFC13
:2074600094F96400BDE83840FBF77EBF38BD00BFE806002038B515460446B8B1016590F923
:207480006400FBF77FFFB4F87630E16E9BB294F865001944064BAAB253F82000FEF7A5FA30
:2074A00094F96400BDE83840FBF75EBF38BD00BFE806002048B1836D013306D190F86520EC
:2074C000024B53F82200FEF757BC7047E806002048B1836D013306D190F86520024B53F88C
:2074E0002200FEF761BC7047E8060020836C04381847C36C0438184730B5044650F804398B
:2075000085B01D6815F0010512D0002200921A6800925B680093009BFFF7ECFE40BB01220D
:20752000204604F1620105B0BDE83040FEF773BC196811F0020106D001951A6801925B68D6
:207540000193019BE8E71A6812F0040206D002911A6802925B680293029BDDE719680907D9
:20756000DAD503921A6803925B680393039BD3E705B030BD08B52520FBF72AFF024B186873
:20758000BDE80840FEF7AEBAE8060020262008B5FBF71EFF034B586818B1BDE80840FEF7C8
:2075A000A1BA08BDE8060020272008B5FBF710FF034B986818B1BDE80840FEF793BA08BD8D
:2075C000E806002003460A4910B508680344EFF30882934205D90C224FF0FF30054B1A6000
:2075E00010BD054A054C121B9342F4D20B60F7E7A800002060090020005000200004000048
:20760000FEE700001622024B4FF0FF301A607047600900200120704710B590B02022002198
:2076200007A800F08DFF1422002101A800F088FF102301220224CDE90A234FF4601306A8E5
:2076400006940D940F93FDF7D3F900B1FEE70F23CDE901344FF480630390CDE904302146D0
:2076600001A8FDF787FB00B1FEE710B010BDB0F80831B0F80421981A00F03F007047B0F8DA
:207680000831B0F804219BB293421ABFD0F8FC30985C4FF0FF30704790F80631B0F80A016A
:2076A000C0B2834227BFC3F13F03C018C01A00F1FF30704707B503688DF8071001225B6885
:2076C0000DF10701984703B05DF804FB13B50DF107010446FFF792FE88B9B4F87430B4F8E3
:2076E0007020013303F03F03934208D0B4F874209DF80700A16E92B28854A4F8743002B0E7
:2077000010BD0000B0F87610826F10B50A4402F03F02A0F87620B0F87610B0F8722089B266
:207720008A421AD0B0F876404032A4B2B0F87610121B544289B204F03F0402F03F02C1F125
:20774000400158BF62428A4228BF0A4604498267FFF790FE4FF0FF3010BD0020FCE700BF73
:20776000057700082DE9F843036804469B6888461646984701232374D4F8EC30B4F80671AD
:2077800001338146C7F1400709D194F8103133B1002304F1940084F81031FFF78BFE2368F1
:2077A00020469B6898470028F9D03546BD4225D84D4523D8B4F80631D4F800015A19402AFF
:2077C000184430D82A46414600F00AFF2F46B4F806311D4405F03F05A4F8065104F19405E2
:2077E0002846FFF799FD30B93A4628461549C4F80C71FFF73FFE3046BDE8F8834F4528BFDD
:207800004F4623683A4641465B6820469847236820469B689847ED1BB844B4F80671814678
:20782000C7F14007C2E7C3F140073A46414600F0D7FED4F80001EA1B08EB070100F0D0FE4E
:20784000C5E700BF05770008C0F8F030009B914208BF4FF0FF31C0F8F43000F11103C0F824
:20786000FC300023C0E93A2100F15102A0F80831C0E94023A0F80A317047000073B54FF49F
:207880007A750026C0E901653D4D069C0560CDB2322D25D83B4E01F4E06156F8255029436A
:2078A000D5B2322D30D8374E02F4E06256F825502A43DDB2322D3BD8324E03F4E06356F8E4
:2078C00025502B43E5B2322D46D82E4E04F4E06456F825502C430094FFF7B6FF02B070BDA9
:2078E00001F0C006C02E0CD1CF2D0AD8264D01F03F0655F82660234D01F4E06155F8265043
:20790000CDE74FF0FF31CBE702F0C006C02E0CD1CF2D0AD81C4D02F03F0655F82660194D58
:2079200002F4E06255F82650C2E74FF0FF32C0E703F0C006C02E0CD1CF2D0AD8124D03F0D8
:207940003F0655F826600F4D03F4E06355F82650B7E74FF0FF33B5E704F0C006C02E0CD186
:20796000CF2D0AD8084D04F03F0655F82660054D04F4E06455F82650ACE74FF0FF34AAE7E1
:20798000049D0008289C0008E89B0008037C70B504460D46A3B1FBF79FFC0646B4F80621A6
:2079A000B4F80A319BB29A420AD0002DF8D0FBF793FC801B8542F1D8B4F80A31A4F8063182
:2079C00070BD0021FFF7E2BFCBB2322B08D80E4A01F4E06152F823301943C0F8EC10704716
:2079E00001F0C002C02A0CD1CF2B0AD8074B01F03F0253F82220044B01F4E06153F82230FE
:207A0000EAE74FF0FF31E8E7289C0008E89B0008CBB2322B08D80E4A01F4E06152F823301B
:207A20001943C0F8E810704701F0C002C02A0CD1CF2B0AD8074B01F03F0253F82220044BCD
:207A400001F4E06153F82230EAE74FF0FF31E8E7289C0008E89B000873B54FF47A73164639
:207A60000022C0E901231D4B044603604FF0FF33C0F8EC301A4B0D46984215D1C321FFF76B
:207A8000A3FFC221FFF7C4FF4FF0FF33012E08BFC4F8EC3000932046D4E93A214FF0FF33E7
:207AA000FFF7D2FE02B070BD0E4B0F499A680F4B53F82200FFF7B2F9854202D1C321204622
:207AC000DDE70B492846FFF7BAF90749C4F8EC002846FFF7B4F9C4F8E800D5E7049D000865
:207AE000F4060020E89B00080C990008289C0008C4980008D0F8EC3010B5013304460ED1FE
:207B00000368DB68984794F8103143B9012304F1940084F81031BDE81040FFF7D9BC10BD58
:207B200073B5144602F00703023BDBB2042B80F8112196BF1A4A0022D25C04F03003302B99
:207B40000546C0F8141107D14FF4C0630132082A09D0092A1BD0FEE714F020031CD04FF428
:207B600080630132F3E70022C4F3C00405F19406640330460094FFF795FB2846FFF7BAFFD4
:207B80003046084902B0BDE87040FFF753BC4FF48052E9E71A46E7E7082AFBD0DBE700BF81
:207BA000F49C0008CD76000810B50446FFF7A2FFB4F80821B4F8043192B29A4217BFD4F8C4
:207BC000FC204FF0FF30D05C01331CBF03F03F03A4F8043110BD0000002202490248FFF760
:207BE0003BBF00BF00440040F406002070B505460C46084649B1F8F789FA2B680246214670
:207C00002846BDE870405B68184770BD08B5FFF7EDFF08BD03681B681847000008B5024999
:207C2000FFF7E4FF08BD00BF8795000838B50546FFF7DCFF04462846FFF7F0FF204438BDC4
:207C4000FFF7F4BF70B50D46144630B1461E012E05D811462846FFF771FB204670BD036833
:207C60005B689847F9E70EB403B503AA52F8041B019200F013FC02B05DF804EB03B0704700
:207C80000023012A98BF0A2230B58BB00C468DF8243009A92546B4FBF2F404FB1253DBB225
:207CA000092B94BF30333733DBB2AA4201F8013DF0D9FFF79BFF0BB030BD2DE9F04107462B
:207CC0000E4614462AB9BDE8F0410368C9B21B6818470A2A05D1002905DBBDE8F041FFF796
:207CE000CFBFD2B2F9E72D21FFF794FF2246054671423846FFF7C4FF2844BDE8F081FFF7A6
:207D0000DCBF10B422B9026810BC1268C9B2104710BCD2B2FFF7B4BFFFF7F3BF38B505460E
:207D2000FFF7EFFF04462846FFF778FF204438BD10B5044600F072FAE060236820465B6981
:207D40009847002808DA00F069FAE368C01AA3689842F2D34FF0FF3010BDF8B507460D4690
:207D60000C468E18B44201D1601BF8BD3846FFF7DFFF431CF8D004F8010BF3E72DE9F04171
:207D80000746884616461D4673B100243846FFF7CFFF431C05D0404503D030550134A54252
:207DA000F4D12046BDE8F0811C46FAE72DE9F041C3B2322B0D46904686B04ED8394A00F42A
:207DC000E06452F823301C43C4F30310FEF7A0FB074600283ED0B8F1020F52D0B8F1030FEF
:207DE00051D0314E314BB8F1000F08BF1E46304B9A6942F001029A619B6903F00103019347
:207E0000019BA4F10D03012B3FD82A4A536823F0E06343F08063536000230122CDE902335F
:207E2000CDE9043304F00F04AB6802FA04F4A4B23BB10222294602A89847EB680593AB68EB
:207E4000049338463346214602AAFEF795FC02A8F8F721FA06B0BDE8F08100F0C002C02ADF
:207E60000CD1CF2B0AD8144B00F03F0253F822200C4B00F4E06453F82230A4E74FF0FF3403
:207E8000A2E70E4EB3E7094EB1E70F2C03D0A4F11303012BC0D8074A536823F0E06343F062
:207EA0000073B8E7289C000800001110000021100010024000000140E89B00080000311033
:207EC00008B50320FBF70EFABDE8084000F0C4B908B5AFF30080F9F7B9FEFAF7CBFA00F042
:207EE000ADF9FAE7C0F30312042A034610B50ED80020084AD9B252F8044B8C4203D103F4E2
:207F0000E063184310BD01303328F4D1FAE73320F8E700BF289C0008FEF7B2FF0B480C49B9
:207F20000C4A002302E0D458C4500433C4188C42F9D3094A094C002301E013600432A242C0
:207F4000FBD300F027FBFFF7C3FF70470000002008010020589D00080801002068090020D2
:207F6000FEE791420FD008D90123891A8B40984208D30130C8400138704720B10130521AAB
:207F80009040F8E700207047014B1860704700BFAC000020C3B2322B2DE9F04107460E469B
:207FA00031D82C4A00F4E06452F823301C43621C4ED020462849FEF749FEDFF8A08005461D
:207FC000002831D0264AC4F3031152F8210004F00F0520FA05F3DB075FBF0123AB40034363
:207FE00042F821301F4BD8F800101D6830462A46FFF7B7FF1C490246EBB22046BDE8F0410F
:208000000968FEF7D9BA00F0C002C02A20D1CF2B1ED8164B00F03F0253F822200D4B00F47F
:20802000E06453F82230C1E73846012100F020F8D8F8001030460822FFF793FF7F2898BF09
:2080400029463846BDE8F04188BF012100F06EB8BDE8F081289C000854990008B400002033
:208060000C080020B0000020AC000020E89B0008C3B2322B2DE9F0410D462AD8274A00F4D2
:20808000E06452F823301C43621C44D0244EC4F3031756F8273004F00F0823FA08F3DB0721
:2080A00010D520461F49FEF7D1FD10B12046FEF7D3FA012256F8273002FA08F223EA020391
:2080C00046F82730052D15D8DFE805F015211B1D1F2300F0C002C02A1DD1CF2B1BD8124BAC
:2080E00000F03F0253F822200C4B00F4E06453F82230C8E7FEE700212046BDE8F041FEF7B0
:20810000B5BD1021F8E72021F6E70321F4E70121F2E70921F0E7BDE8F08100BF289C000823
:208120000C08002054990008E89B0008C3B2322B1BD8174A00F4E06052F823301843431CDA
:2081400025D0C0F30313042B98BF124A00F00F0098BF52F82320104B88BF002253F820303D
:20816000C3F30F2391B11361704700F0C002C02A0DD1CF2B0BD8094B00F03F0253F8222041
:20818000034B00F4E06053F82230D7E753617047289C00080C000020F4970008E89B000881
:2081A000C3B2322B1CD8194A00F4E06052F823301843431C25D0C0F30313042B23D8144AC5
:2081C00000F00F0052F82330124A9B6852F82020D84300EA122080B2B0FA80F04009704797
:2081E00000F0C002C02A0CD1CF2B0AD80A4B00F03F0253F82220054B00F4E06053F82230F6
:20820000D6E70020704700239B68FFDE289C00080C000020F4970008E89B0008FEF748BABA
:2082200038B5044648B1FEF743FA054600F016F8FEF73EFA431BA342F8D338BD08B5044B57
:208240002BB10448FFF713FA08B1AFF3008008BD00000000F4060020FEF776BA704700005D
:20826000024B0146186800F02DB800BFB8000020024B0146186800F0C1B900BFB800002069
:2082800070B50F4E0C463168054611B900F060F930602146284600F05BF9431C03D14FF0F8
:2082A000FF34204670BDC41C24F00304A042F8D0211A284600F04CF90130F2D1EFE700BFEC
:2082C000200800202DE9F843CD1C25F0030508350C2D38BF0C25002D064601DBA94204D944
:2082E0000C2333600020BDE8F883DFF8D48000F069F8D8F800301C4644BB29463046FFF7C4
:20830000BFFF431C044658D1D8F800402746002F43D1002C4BD023683946304604EB03094B
:2083200000F016F9814542D1216830466D1A2946FFF7A6FF01303AD023682B442360D8F84D
:2083400000305A6862BBC8F800700FE02268521B20D40B2A17D96119A342256018BF59606B
:20836000636808BFC8F8001062514B60304600F02FF804F10B00231D20F00700C21A1CBFA2
:208380001B1AA350AFE76268A3420CBFC8F800205A60EBE723466468AEE73C467F68B6E769
:2083A0001A465B68A342FBD100235360DEE70C233046336000F00CF894E70560D6E700BFC6
:2083C00024080020014800F009B900BF64090020014800F004B900BF64090020024B0A462B
:2083E0000146186800F002B8B80000202DE9F041074614460D4621B91146BDE8F041FFF7F6
:2084000061BF2AB900F0FAF825462846BDE8F08100F03CF98442064602D8B4EB500FF4D8AD
:2084200021463846FFF74EFF804608B94546ECE7B4422246294628BF324600F0D1F82946DB
:20844000384600F0DBF8F1E72DE9F0410F464FF40071ADF5047D03AD0DF1100829600093AE
:20846000414613462A46064600F022F8044688B10246394630462B6800F07AF84445286090
:2084800003D02146304600F0B9F828680DF5047DBDE8F0814FF0FF30F8E7000013460A466C
:2084A000014602480068FFF7CFBF00BFB800002070B515469AB01A4689B12C689CB94FF418
:2084C000227321460026B442ADF80C301996009104910BDA8B23036000201AB070BD4FF47E
:2084E00022730C46EEE74FF4C163EBE74FF6FF736946ADF80E301E9B0294059400F02EF93F
:208500000028E9DB009B28601E700498E5E7884210B501EB020402D98442234607D8431E8B
:20852000A14207D011F8012B03F8012FF8E70244824200D110BD13F8011D02F8011DF7E77B
:2085400003460244934200D1704703F8011BF9E738B50023054D044608462B60FFF732F893
:20856000431C02D12B6803B1236038BD6009002038B50446084611460022054D2A601A4647
:20858000FFF760FB431C02D12B6803B1236038BD6009002070B500260C4D0D4B5B1B9C10F2
:2085A000A64209D1002600F0C5FB0A4D0A4B5B1B9C10A64205D170BD55F8043B98470136C8
:2085C000EEE755F8043B98470136F2E7309D0008309D0008309D0008489D00087047704771
:2085E0000A44914200F1FF3300D1704710B511F8014B914203F8014FF9D110BD38B50546A8
:20860000002940D051F8043C0C1F002BB8BFE418FFF7D8FE1C4A136833B963601460284691
:20862000BDE83840FFF7D4BEA34208D9206821188B4201BF19685B6809182160EDE71A4667
:208640005B680BB1A342FAD911685018A0420BD120680144501883421160E0D118685B68E5
:20866000084410605360DAE702D90C232B60D6E7206821188B4201BF19685B680918216044
:2086800063605460CBE738BD2408002051F8043C181F002BBCBF0B58C01870472DE9F047CB
:2086A0001F468E688246BE420C469046334653D8B1F90C0010F4906F2BD06569236809694C
:2086C00005EB4505A3EB010905EBD5757B1C6D104B44AB422A4684BF1D462A46430527D534
:2086E00011465046FFF7EEFD064658B34A462169FFF776FFA38923F4906343F08003A381C0
:2087000026614E4426603B463E466561A5EB0905A5601F463A4641462068FFF7F8FE00204C
:20872000A3689B1BA36023683B442360BDE8F0875046FFF75BFE06460028E1D150462169A1
:20874000FFF75CFF0C23CAF80030A3894FF0FF3043F04003A381E9E73E46DBE72DE9F04F08
:2087600098468B8907461B060D4614469DB010D50B6973B94021FFF7A5FD2860286130B927
:208780000C233B604FF0FF301DB0BDE8F08F40236B610023099320238DF8293030234FF00F
:2087A0000109CDF80C80DFF898818DF82A3023469A4613F8012B0AB1252AF9D1BAEB040B87
:2087C0000BD05B46224629463846FFF767FF013000F0A780099A5A4409929AF80030002B5B
:2087E00000F09F8000234FF0FF32CDE905230AF1010A049307938DF853301A93544605224C
:2088000014F8011B4E4800F037FA049AD8B9D00644BF20238DF85330110744BF2B238DF838
:2088200053309AF800302A2B15D0544600204FF00A0C079A214611F8013B303B092B4BD99A
:20884000B0B1079214E0A0EB080309FA03F31343A2460493D2E7039B191D1B680391002BF7
:20886000BBBF5B4242F0020207930793B8BF049223782E2B0AD163782A2B32D1039B023494
:208880001A1D1B68039243EAE3730593DFF8B4A003225046217800F0EFF938B14022049B2D
:2088A000A0EB0A00824013430134049314F8011B062225488DF8281000F0DEF9002836D0D0
:2088C000224B1BBB039B073323F0070308330393099B334409936AE70C4601200CFB0232D9
:2088E000A8E700234FF00A0C194601340593204610F8012B303A092A03D9002BC6D00591DB
:20890000C4E7044601230CFB0121F0E703AB00932A4638460E4B04A9AFF30080421C06463D
:20892000D6D1AB895B063FF52DAF09982CE703AB00932A463846064B04A900F07DF8EDE7D1
:208940008A9500089095000894950008000000009D8600082DE9F047164698468A680B697A
:2089600007469342B8BF1346336091F843200C46DDF820900AB1013333602368990642BF02
:20898000336802333360256815F0060506D104F1190AE36832689B1AAB422BDC94F843305B
:2089A0002268003B18BF0123920630D44146384604F14302C847013023D02368226903F0E0
:2089C0000603042B14BF002533684FF0000608BFE56804F11A0408BFED1A54F8123C08BF31
:2089E00025EAE5759342C4BF9B1AED18B5421AD1002008E00123524641463846C847013011
:208A000003D14FF0FF30BDE8F0870135C1E73020E11881F843005A1C94F845102244023323
:208A200082F84310C2E70123224641463846C8470130E6D00136D9E72DE9FF470F7E914682
:208A4000782F80460C469A460C9E01F1430207D8622F0AD8002F00F0D280582F00F0B78025
:208A600004F1420684F842703AE0A7F16303152BF6D801A151F823F0D18A0008E58A00088D
:208A8000618A0008618A0008618A0008618A0008E58A0008618A0008618A0008618A0008BA
:208AA000618A0008E58B00080F8B00089B8B0008618A0008618A0008078C0008618A000807
:208AC0000F8B0008618A0008618A0008A38B000833681A1D1B68326004F1420684F84230C6
:208AE00001239DE033682068191D3160060601D51D6803E04506FBD5B3F90050002D03DA80
:208B00002D236D4284F843300A23594810E021683368080653F8045B02D4490648BFADB242
:208B20006F2F5348336059D10823002184F843106668002EA66005DB21682E4321F0040132
:208B400021604DD01646B5FBF3F103FB1157C75D06F8017D2F46BB420D46F4D9082B0BD1E0
:208B60002368DF0708D5236961689942DEBF302306F8013C06F1FF36921B22614B462146F8
:208B80004046CDF800A003AAFFF7E4FE01304CD14FF0FF3004B0BDE8F087236843F02003F8
:208BA00023607827334884F84570236831681F0651F8045B02D45F0648BFADB23160D907E4
:208BC00044BF43F0200323601DB11023ADE72848E9E7236823F020032360F6E70A23A4E70B
:208BE0001646BBE733682568181D616930602E061B6801D5196002E06806FBD519800023DE
:208C000016462361BAE7336800211A1D32601E686268304600F030F808B1801B6060636891
:208C20002361002384F84330A8E73246494640462369D0470130ABD023689B0713D4E068D7
:208C4000039B9842B8BF1846A4E70123324649464046D04701309BD00135E36803995B1A46
:208C6000AB42F2DCEBE7002504F11906F5E700BF9B950008AC950008034610B5C9B2024443
:208C80009342184601D1002003E0047801338C42F6D110BD062008B500F02CF80120FEF7AD
:208CA000AFFC1F2938B505460C4604D9162303604FF0FF3038BDC26B12B152F821304BB9CC
:208CC000284600F031F8224601462846BDE8384000F018B8012B0AD0591C03D11623036028
:208CE0000120E7E70021204642F8241098470020E0E70000024B01461868FFF7D2BF00BF70
:208D0000B800002038B50023064D0446084611462B60FEF777FC431C02D12B6803B123603A
:208D200038BD00BF60090020FEF774BC08B5FFF7B1FF0000F8B500BFF8BC08BC9E467047EF
:208D4000F8B500BFF8BC08BC9E4670477E58506F7765727341585032313031005344413A7F
:208D600025642053434C3A2564004865616450686F6E65206465746563746564004D6973AE
:208D800074616B65202120546865207374657073206973206D757374202575206D56004D8E
:208DA000697374616B65202120546865206D696E696D756D207365747461626C6520766F1B
:208DC0006C74616765206F662056535953206973202575206D56004D697374616B65202174
:208DE00020546865206D6178696D756D207365747461626C6520766F6C74616765206F6699
:208E00002056535953206973202575206D56004661696C656420746F2064697361626C6508
:208E20002074686520706F776572206368616E6E656C2C2074686520706F776572206368C6
:208E4000616E6E656C20686173206265656E2070726F74656374656400454E41424C45005D
:208E600044495341424C45002573202D204845583A30782578200A004D697374616B65207D
:208E8000212020546865207374657073206973206D7573742025756D56004D697374616B36
:208EA00065202120546865207374657073206973206D7573742025756D56004D697374611C
:208EC0006B65202120444335206D696E696D756D20766F6C746167652069732025756D56FE
:208EE000202C25756D56004D697374616B65202120444335206D6178696D756D20766F6C4F
:208F0000746167652069732025756D56004D697374616B65202120424C444F31206D696E52
:208F2000696D756D206F757470757420766F6C74616765206973202025756D56004D6973D4
:208F400074616B65202120424C444F31206D6178696D756D206F757470757420766F6C74E5
:208F6000616765206973202025756D56004D697374616B65202120444C444F31206D696E44
:208F8000696D756D206F757470757420766F6C74616765206973202025756D56004D697374
:208FA00074616B65202120444C444F31206D6178696D756D206F757470757420766F6C7483
:208FC000616765206973202025756D56004D697374616B65202120427574746F6E2062613D
:208FE0007474657279206368617267696E67207374657020766F6C746167652069732025A7
:2090000075206D56004D697374616B65202120546865206D696E696D756D20636861726767
:2090200065207465726D696E6174696F6E20766F6C74616765206F662074686520636F693E
:209040006E2063656C6C2062617474657279206973202575206D56004661696C6564207455
:209060006F207365742074686520706F776572206368616E6E656C2C2074686520706F776B
:209080006572206368616E6E656C20686173206265656E2070726F746563746564004D694A
:2090A0007374616B65202120444331206D696E696D756D20766F6C74616765206973202510
:2090C00075206D56004D697374616B65202120444331206D6178696D756D20766F6C7461ED
:2090E0006765206973202575206D56004D697374616B65202120414C444F31206D696E69BE
:209100006D756D206F757470757420766F6C74616765206973202025756D56004D697374E7
:20912000616B65202120414C444F31206D6178696D756D206F757470757420766F6C746117
:209140006765206973202025756D56004D697374616B65202120414C444F32206D696E695C
:209160006D756D206F757470757420766F6C74616765206973202025756D56004D69737487
:20918000616B65202120414C444F32206D6178696D756D206F757470757420766F6C7461B6
:2091A0006765206973202025756D56004D697374616B65202120414C444F33206D696E69FB
:2091C0006D756D206F757470757420766F6C74616765206973202025756D56004D69737427
:2091E000616B65202120414C444F33206D6178696D756D206F757470757420766F6C746155
:209200006765206973202025756D56004D697374616B65202120414C444F34206D696E6999
:209220006D756D206F757470757420766F6C74616765206973202025756D56004D697374C6
:20924000616B65202120414C444F34206D6178696D756D206F757470757420766F6C7461F3
:209260006765206973202025756D56004D697374616B652021204350554C444F206D696E2F
:20928000696D756D206F757470757420766F6C74616765206973202025756D56004D697371
:2092A00074616B652021204350554C444F206D6178696D756D206F757470757420766F6C81
:2092C00074616765206973202025756D5600504D55206973206E6F74206F6E6C696E652E22
:2092E0002E2E0067657449443A307825780A00594553004E4F0069734368617267696E672F
:209300003A0069734469736368617267653A0069735374616E6462793A006973566275730C
:20932000496E3A00697356627573476F6F643A00676574436861726765725374617475737D
:209340003A007472695F636861726765007072655F63686172676500636F6E7374616E7441
:209360002063686172676500636F6E7374616E7420766F6C7461676500636861726765205D
:20938000646F6E65006E6F74206368617267696E0067657442617474566F6C746167653A03
:2093A0000067657456627573566F6C746167653A0067657453797374656D566F6C7461678F
:2093C000653A006765744261747465727950657263656E743A002500535441545553203D62
:2093E0003E204845583A002042494E3A00697344726F705761726E696E674C6576656C324C
:2094000000697344726F705761726E696E674C6576656C3100697357647454696D656F755E
:20942000740069734261744368617267654F76657254656D70657261747572650069734233
:209440006174576F726B4F76657254656D7065726174757265006973426174576F726B557F
:209460006E64657254656D706572617475726500697356627573496E736572740069735692
:2094800062757352656D6F7665006973426174496E7365727400697342617452656D6F76B0
:2094A0006500697350656B657953686F72745072657373005265616420706D752064617409
:2094C0006120627566666572202E002C00697350656B65794C6F6E675072657373006973C4
:2094E00050656B65794E6567617469766500697350656B6579506F73697469766500697332
:209500004C646F4F76657243757272656E744972710069734261746665744F7665724375FB
:209520007272656E74497271006973426174436861676572446F6E65006973426174436873
:209540006167657253746172740069734261744469654F76657254656D7065726174757294
:20956000650069734368616765724F76657254696D656F75740069734261744F76657256F8
:209580006F6C74616765000D0A00232D302B2000686C4C006566674546470030313233344F
:2095A0003536373839414243444546003031323334353637383961626364656600000000A1
:2095C000000000000000000017080008A30A00087907000887070008350800081902000829
:2095E000390200085D0300085D01000815120008D91000087D0A0008CB080008750800084B
:20960000AD11000851130008A90700085B09000891190008293200083732000847320008ED
:20962000E1310008D11E0008CB1500084B090008EB1E000859120008250900089715000867
:209640001509000863150008FF0800088908000823120008F5140008E9140008B3010008AD
:20966000C9010008870100089D0100085F01000871010008DF010008F501000859110008A8
:2096800043130008671100083513000883110008271300089F110008191300087511000844
:2096A0000B13000891110008FD1200087510000833150008E908000801150008D9080008E6
:2096C0000000020000050000030000043029003928005D7D005B7B00B70000B5D600B6D743
:2096E00000B40000859000848900838800828700818600607E00332300324000080000D4F7
:20970000D500C1000009D200B1D0003424004500005700005000003D2B002D5F005C7C0047
:209720002F3F005200005300003121000AD100382A00372600365E0035250046000058009E
:20974000005100002E3E004900005500005900005400005600003B3A004100004C00004B5E
:2097600000004A00004800004700004300002722005A00004F00002C3C004D00004E0000D8
:20978000420000440000200000000000C8C91213141516171C1D1E1FCACBCCCDCECF262789
:2097A000C0C1C2C3C4C5C60000000000000000009F290008E12900088D2600083D2B000847
:2097C0009126000899260008B32600085B7D00087D7D0008010202030405060708090A0BFC
:2097E0000C0D0E0F1010020104030204081004004000000401010000020200000404000095
:2098000008080000101000002020000040400000808000000100010402000204040004043E
:2098200008000804100010042000200440004004800080040000000001020304000000001A
:209840000000000001020304060708090000000000440040120000000B00000000380140C6
:20986000120000001D00000000480040120B00001D01000000480040120A0000FFFFFFFF56
:2098800000000000000000000100000000440040120800000C000000003801401200000092
:2098A0001E00000000480040120000001E01000000480040120A0000FFFFFFFF0000000031
:2098C000000000000300000000440040100800000A00000000380140100600001700000039
:2098E00000380140100500001B00000000480040100000002B00000000480040100A00005A
:20990000FFFFFFFF0000000000000000020000000044004012080000090000000038014029
:20992000120600001600000000380140120500001A00000000480040120000002A0000008B
:2099400000480040120A0000FFFFFFFF000000000000000000000000000000401280000095
:2099600000010000000000401290000001000000000000401212010001010000000000405C
:209980001210010002000000000000401292010002010000000000401291010003000000D3
:2099A0000000004012120200030100000000004012110200060000000004004012950000E7
:2099C00007000000002C0140128D100007010000000400401215010008000000002C01407B
:2099E000128E000008010000002C0140128D000009000000002C0140120E01000901000011
:209A0000002C0140120D01000A000000002C0140128E01000A010000002C0140128D010089
:209A20000B000000002C0140120E02000B010000002C0140120D02000F00000000000040A3
:209A4000129100000F01000000000040128F000010000000002C0140120D110010010000B4
:209A6000000400401295010010020000000400401294010011000000002C0140128D1100CF
:209A8000110100000004004012150200110200000004004012140200130000000000004075
:209AA000121101001301000000000040120F010014000000000400401294000015000000F9
:209AC00000040040121401001600000000080040129700001700000000080040121701008B
:209AE0001800000000080040129701001900000000080040121702001A0000000000004076
:209B0000129001001A01000000000040128F01001B00000000000040121002001B0100000A
:209B200000000040120F02001D000000002C0140128E10001E000000002C0140120E1100CC
:209B40001F000000002C0140128E110026000000000400401293000027000000000400404E
:209B600012130100280000000004004012930100290000000004004012130200FFFFFFFF1D
:209B8000000000000000000016000000005400400A04000018000000005400400A03000054
:209BA0001A000000005800400A000000FFFFFFFF0000000000000000170000000054004042
:209BC0000A04000019000000005400400A0300001B000000005800400A000000FFFFFFFF04
:209BE000000000000000000000000000010000000200000003000000040000000500000056
:209C0000060000000700000010000000110000002000000021000000220000002300000090
:209C20002400000025000000000000000100000002000000030000000400000005000000CC
:209C4000060000000700000008000000090000000A0000000B0000000C0000000D000000B8
:209C60000E0000000F00000010000000110000001200000013000000140000001500000058
:209C8000160000001700000018000000190000001A0000001B0000001C0000001D000000F8
:209CA0001E0000001F00000020000000210000002200000023000000240000002500000098
:209CC000260000002700000028000000290000002A0000002B0000002C0000002D00000038
:209CE0002E0000002F0000003000000031000000320000000600070008000000000000005F
:209D000000000000B57600086577000899760008C37900086F760008A97B00087F760008BB
:209D20005B7D00087D7D0008E463FF7F01000000C17E0008410100088D240008D12C00082C
:209D400009690008D97B00081D010008E5240008E12C0008E16900081428506EFF01000095
:209D60001000000000080140000C01400010014000140140001801400030024000000000CC
:209D800000127A000000000000000000000000000000000000000000000000000000000037
:209DA0000000000000000000000000000000000000000000000000000000000000000000A3
:209DC000000000000000000000000000000000000000000000000000FFFFFFFFFFFFFFFF8B
:209DE000FFFFFFFFFFFFFFFF00030000000000000000000000000000000000000000000068
:209E000068090020E80300000800000008000000BC000020000000002808002090080020D2
:209E2000F80800200000000000000000000000000000000000000000000000000000000002
:209E4000000000000000000000000000000000000000000000000000000000000000000002
:209E6000FFFFFFFFFFFFFFFFFFFFFFFFFFFFFFFFFFFFFFFFFFFFFFFFFFFFFFFFFFFFFFFF02
:209E8000FFFFFFFFFFFFFFFFFFFFFFFFFFFFFFFFFFFFFFFFFFFFFFFFFFFFFFFFFFFFFFFFE2
:209EA000FFFFFFFFFFFFFFFFFFFFFFFFFFFFFFFFFFFFFFFFFFFFFFFFFFFFFFFFFFFFFFFFC2
:00000001FF
